:020000040800F2
:10000000D8FF0120E91E000821130008231300086F
:10001000251300082713000829130008000000001A
:100020000000000000000000000000002B1300088A
:100030002D130008000000002F13000831130008E2
:10004000391F0008391F0008391F0008391F000830
:10005000391F0008391F000833130008391F000832
:10006000391F0008391F0008391F0008391F000810
:10007000391F0008391F0008391F0008391F000800
:10008000391300084513000851130008391F0008F0
:10009000391F0008391F0008391F0008391F0008E0
:1000A000391F00085D130008391F0008391F0008B8
:1000B000691300087513000881130008391F000830
:1000C000391F0008391F0008391F0008391F0008B0
:1000D000391F0008391F00088D130008391F000858
:1000E00099130008391F0008391F0008D1130008B0
:1000F000DD130008E1130008E5130008391F0008AC
:10010000391F0008391F0008E9130008391F0008CB
:10011000391F0008391F0008391F0008391F00085F
:10012000F5130008391F0008391F0008391F00089F
:10013000391F00080000000000000000391F0008FF
:10014000391F0008391F0008391F00080114000872
:10015000391F0008391F0008391F0008391F00081F
:10016000391F0008391F0008391F0008391F00080F
:10017000391F0008391F0008391F0008000000005F
:1001800000000000391F000800000000000000000F
:10019000391F00080000000000000000391F00089F
:1001A000000000000000000000000000391F0008EF
:1001B000391F0008391F0008391F0008391F0008BF
:0401C000391F0008DB
:1001C40010B5054C237833B9044B13B10448AFF38D
:1001D40000800123237010BD1401002000000000E2
:1001E400207D000808B5034B1BB103490348AFF356
:1001F400008008BD0000000018010020207D0008D8
:10020400034613F8012B002AFBD1181A0138704752
:1002140053B94AB9002908BF00281CBF4FF0FF3169
:100224004FF0FF3000F074B9ADF1080C6DE904CE65
:1002340000F006F8DDF804E0DDE9022304B07047BD
:100244002DE9F047089D04468E46002B4DD18A4285
:10025400944669D9B2FA82F252B101FA02F3C2F1B8
:10026400200120FA01F10CFA02FC41EA030E944049
:100274004FEA1C48210CBEFBF8F61FFA8CF708FB6A
:1002840016E341EA034306FB07F199420AD91CEB42
:10029400030306F1FF3080F01F81994240F21C8174
:1002A400023E63445B1AA4B2B3FBF8F008FB1033BC
:1002B40044EA034400FB07F7A7420AD91CEB0404F1
:1002C40000F1FF3380F00A81A74240F207816444C1
:1002D400023840EA0640E41B00261DB1D440002346
:1002E400C5E900433146BDE8F0878B4209D9002DAA
:1002F40000F0EF800026C5E9000130463146BDE834
:10030400F087B3FA83F6002E4AD18B4202D382429D
:1003140000F2F980841A61EB030301209E46002D4C
:10032400E0D0C5E9004EDDE702B9FFDEB2FA82F2A1
:10033400002A40F09280A1EB0C014FEA1C471FFAFF
:100344008CFE0126200CB1FBF7F307FB131140EAE6
:1003540001410EFB03F0884208D91CEB010103F1B3
:10036400FF3802D2884200F2CB804346091AA4B275
:10037400B1FBF7F007FB101144EA01440EFB00FE49
:10038400A64508D91CEB040400F1FF3102D2A645AE
:1003940000F2BB800846A4EB0E0440EA03409CE74D
:1003A400C6F12007B34022FA07FC4CEA030C20FAFA
:1003B40007F401FA06F31C43F9404FEA1C4900FA1A
:1003C40006F3B1FBF9F8200C1FFA8CFE09FB181197
:1003D40040EA014108FB0EF0884202FA06F20BD90A
:1003E4001CEB010108F1FF3A80F08880884240F25A
:1003F4008580A8F102086144091AA4B2B1FBF9F09E
:1004040009FB101144EA014100FB0EFE8E4508D998
:100414001CEB010100F1FF346CD28E456AD902381D
:10042400614440EA0840A0FB0294A1EB0E01A14202
:10043400C846A64656D353D05DB1B3EB080261EB70
:100444000E0101FA07F722FA06F3F1401F43C5E94A
:10045400007100263146BDE8F087C2F12003D84080
:100464000CFA02FC21FA03F3914001434FEA1C47C2
:100474001FFA8CFEB3FBF7F007FB10360B0C43EAB4
:10048400064300FB0EF69E4204FA02F408D91CEB64
:10049400030300F1FF382FD29E422DD90238634462
:1004A4009B1B89B2B3FBF7F607FB163341EA034102
:1004B40006FB0EF38B4208D91CEB010106F1FF3851
:1004C40016D28B4214D9023E6144C91A46EA004648
:1004D40038E72E46284605E70646E3E61846F8E6DA
:1004E4004B45A9D2B9EB020864EB0C0E0138A3E723
:1004F4004646EAE7204694E74046D1E7D0467BE704
:10050400023B614432E7304609E76444023842E77B
:10051400704700BF7FB5134C1348009405254FF472
:1005240080561023CDE901561A46A02102F002FE9E
:1005340010B1012004B070BD322001F029FDCDE9D5
:1005440001561023094D084800951A46A02102F0CF
:1005540081FE0028EDD1A878A378C01A18BF012025
:10056400E8E700BF000000207002002030010020F6
:1005740007B5222001F050FC01F044FC019001F089
:100584006FFC019803B05DF804FB000010B5064C45
:1005940001F06EFC18B1BDE81040FFF7E9BF013C63
:1005A400F6D1FA2010BD00BF404B4C0008B501F055
:1005B40033FC01F055FCBDE80840FFF7E7BF08B580
:1005C40001F056FC08B1FFF7D3FFBDE80840302026
:1005D400FFF7ECBF1FB510220021684607F080FB2F
:1005E4003548364A0023C0E90023354A8262012493
:1005F400072283600461047680F82030C362C360FC
:10060400C26180F83040436101F0D6FC08B100F0CB
:100614002DFD0823CDE900342748072369460293BA
:1006240001F02AFF08B100F021FD4FF0090E02236A
:1006340021486946CDE900E301F01EFF08B100F04E
:1006440015FD4FF00A0C03231B486946CDE900C38E
:1006540001F012FF08B100F009FD0B240423164831
:100664006946CDE9004301F007FF08B100F0FEFC44
:100674000C200523CDE9000369460F4801F0FCFE78
:1006840008B100F0F3FC0D210623CDE900130A485C
:10069400694601F0F1FE08B100F0E8FC0F220723DF
:1006A40005486946CDE9002301F0E6FE08B100F0F3
:1006B400DDFC04B010BD00BF380100200020014063
:1006C4000100000F70B5064688B01422002103A86B
:1006D40007F006FB32682B4B9A4251D103F58C3359
:1006E400002500955A6C284842F480725A645A6C6A
:1006F40002F480720092009A01951A6B42F004028F
:100704001A631A6B02F004020192019A02951A6BA1
:1007140042F002021A631B6B03F0020302930324E8
:10072400029B03A92F23CDE9033402F08BF9174868
:10073400059503A9CDE9034402F084F9144C154B43
:100744004FF48062C4E900354FF48053C4E90423B4
:1007540020464FF48043C4E90255C4E90635C4E990
:10076400085501F0A1FF08B100F080FC0022B46339
:1007740012201146A66301F02FFF122001F05EFF44
:1007840008B070BD0020014000080240000402408F
:1007940080010020106402400268054B9A4205D192
:1007A400044B054801221A7001F056BD704700BF82
:1007B40000200140E001002038010020A823584314
:1007C400800800BF0138FCD270470000094B48F292
:1007D40015214AF25A52598052211A809980064BA7
:1007E4001A8048F204325A8051229A8010229A7157
:1007F400704700BF580200202802002070B50C4B3F
:1008040086B06A4603F118061546186859681446F6
:1008140003C40833B3422246F7D1182229460548B7
:1008240005F0EEF8052001F0B3FB06B070BD00BF83
:10083400580200204806002007B50A4B18689A8819
:1008440000909B79ADF804206946072206488DF88C
:10085400063005F0D5F8052001F09AFB03B05DF8E9
:1008640004FB00BF280200204806002008B5FFF75B
:10087400ADFF01F009FBFFF74DFE054B0002D882E6
:1008840001F032F901F036F9BDE8084001F038B959
:10089400580200202DE9F74F5D4B1A78012A03D145
:1008A40000221A70FFF7C8FF5A4B1B78012B40F047
:1008B400AC80594D2B785A2B76D1AB78242B73D13D
:1008C400B5F80720554BB5F8116052BA1A811FFAD2
:1008D40082FEB5F8092052BA5A811FFA82FCB5F893
:1008E4000B2052BA9A8197B2B5F80D2052BA90B241
:1008F40076BA0190DA81E87CEA7B5E82B4B22E7D1E
:1009040040EA022246EA0020B5F815601A8276BA57
:10091400DE821FFA86FAB5F81760988276BA1E83CB
:100924001FFA86F9B5F8196076BA5E831FFA86F85D
:10093400B5F81B6076BA9E83B5F81D6076BADE837F
:10094400B5F81F6076BA1E84B5F82160002176BA26
:10095400196059605E84B5F82360B5F825506DBA06
:1009640076BA1FFA85FB9E84DD842D4E2D4DBBF196
:10097400000F27D1336801995863C3F838A0C3F82E
:100984003C90C3F840802B68C3F834E0C3F838C007
:10099400DF631964244B1B689A63DC6301F0B6F8C7
:1009A40001F0EAF801F01CF91A4A1B491F48002318
:1009B4001370272205F016FB052003B0BDE8F04FA5
:1009C40001F0E6BA1846282207F08AF9184A127884
:1009D400012A18BF4FF6FF728283C283028401F09A
:1009E40095F801F0C9F801F0FBF83268322353633B
:1009F4009363D36313642A6853639363D363136465
:100A0400094A12689363D363CEE703B0BDE8F08F5D
:100A14000800002006000020000200203002002010
:100A24005C040020A40400203405002048060020B3
:100A34000700002038B526490B78012B47D1254BF8
:100A44001A78012A43D1244C244D00220A701A70CA
:100A5400234B2268C2F3072103EA02220A442A82B2
:100A64006268C2F3072103EA02220A446A82A26886
:100A7400C2F3072103EA02220A44EA80E268C2F3CD
:100A8400072103EA02220A442A812269C2F30721C8
:100A940003EA02220A446A816269C2F3072103EA73
:100AA40002220A44A169AA8103EA0123C1F30722AD
:100AB4001344EB8101F00FFA0002A8822146094891
:100AC400072201F01FFBBDE83840FFF797BE38BD91
:100AD400E001002008000020E4010020580200206A
:100AE40000FFFF0038010020034B1B780BB9FFF710
:100AF400A1BFFFF7CFBE00BF27020020064B074A65
:100B0400D3F8FC1F914206D10022C3F8FC2FA3F5B1
:100B14003C335B681847704700F00120EFBEADDE40
:100B2400024B034AC3F8FC2F01F096BD00F00120EC
:100B3400EFBEADDE07B5184B00220092196B41F4ED
:100B440080011963196B01F48001009100990192ED
:100B5400196B41F4001119631B6B03F40013114664
:100B640001931020019B01F037FD102001F066FD78
:100B740000221146112001F02FFD112001F05EFD2D
:100B840000221146382001F027FD382003B05DF81B
:100B940004EB01F053BD00BF003802402DE9F04FD3
:100BA4008DB01422002107A807F09AF80024704B96
:100BB40001941A6B6F4F704EDFF8C4A142F010021B
:100BC4001A631A6B02F010020192019A02941A6BD2
:100BD40042F004021A631A6B02F004020292029AAF
:100BE40003941A6B42F080021A631A6B02F08002BB
:100BF4000392039A04941A6B42F001021A631A6B6B
:100C040002F001020492049A05941A6B42F0020263
:100C14001A631A6B02F002020592059A06941A6B83
:100C240042F008021A631B6B03F008030693224682
:100C3400384648F27F01069B01F0DEFF224630462B
:100C440048F2121101F0D8FF2246504640F2044106
:100C540001F0D2FF494B2246184640F6FF710125A8
:100C640001F0CAFF48F27F0207A93846A7F50067DA
:100C74004FF44418CDE90725CDE9094401F0E2FE1B
:100C84004FF4784207A93846CDE90728099401F0C2
:100C9400D9FE07A93046CDE90758099501F0D2FEDF
:100CA40048F2021207A93046CDE907254FF0100992
:100CB400CDE9094401F0C6FE07A93046CDE9079500
:100CC400CDE9095401F0BEFE07A93846CDE90794E1
:100CD4004FF0020B099501F0B5FE042207A9504616
:100CE400CDE907254FF48069CDE909B401F0AAFEE6
:100CF40007A95046CDE90795CDE9094401F0A2FEC4
:100D04001E4B40F6FF7207A91846CDE90725CDE929
:100D1400094401F097FE4FF40073CDE9073B07A99E
:100D24000F2330460B93CDE9094401F08BFE07A94C
:100D34003046CDE90794099401F084FE07A93846AA
:100D4400CDE90798099501F07DFE2246214606204B
:100D540001F042FC062001F071FC224621462820C5
:100D640001F03AFC282001F069FC0DB0BDE8F08FD9
:100D7400003802400010024000000240000C024013
:100D84000004024008B50B480B4A0C4BC0E9002391
:100D940000234FF48042C0E90233C0E90423C0E9D0
:100DA4000633036202F01EF918B1BDE8084000F0F2
:100DB4005DB908BD7002002000540040A086010007
:100DC40030B5044689B01422002103A806F088FF38
:100DD4002268134B9A4221D1124C134800250195E5
:100DE400236B43F002032363236B03F00203019399
:100DF400019BC0221223CDE9032302210423CDE960
:100E0400061303A901F01EFE0295236C43F400139C
:100E14002364236C03F400130293029B09B030BDD6
:100E240000540040003802400004024030B595B040
:100E34001022002109A806F053FF1422002102A861
:100E440006F04EFF204B002100911A6C42F08052B4
:100E54001A641B6C1D4A03F080530093009B01919C
:100E6400136823F4404343F480431360136803F48A
:100E740040430193019B01224FF480330224CDE9C6
:100E840007234FF48003CDE90D43062148230325AE
:100E940007A8CDE90F13CDE91254119403F09EFB7A
:100EA40008B172B6FEE70F23CDE902354FF4805343
:100EB400CDE905300490214602A803F05FF808B19B
:100EC40072B6FEE715B030BD003802400070004035
:100ED4007FB5FFF713FE01F02FF8FFF7A7FFFFF729
:100EE4005DFEFFF727FEFFF775FB00F02FFC00F017
:100EF40095FC00F0FBFC00F0BBF800F0FFF800F0FC
:100F0400D9F800F0C1FAFFF73DFF06F061FC00F0EC
:100F14009BFE00F0EBFA2F4804F002F92E4804F08F
:100F2400FFF82E4804F0FCF82D4804F0F9F82D4899
:100F340004F0F6F82C4A10685168128903AB03C315
:100F4400002125481A8004F039FC0421224804F0C9
:100F540035FC0821204804F031FC0C211E4804F023
:100F64002DFC00211D4804F029FC04211B4804F039
:100F740025FC0821194804F021FC0C21174804F031
:100F84001DFC0421174804F019FC0821154804F03D
:100F940015FC16491648072201F0B4F84FF6FF7302
:100FA4000A2203A9134803F0E7FD4FF6FF730A2250
:100FB40003A9104803F082FF4FF6FF7303AA0093BE
:100FC40011460A230B4803F085FEFFF74FFCFFF799
:100FD4008BFDFCE7140400205C040020A404002022
:100FE400EC04002034050020517D0008E4010020B9
:100FF40038010020C40200200268154B9A4210B543
:10100400044601D100F0B2FF2368B3F1804F14D13C
:10101400104B1B681BB11048022101F0F2FD0F4B6D
:101024001B681BB10C48102101F0EBFD0C4B1B6835
:101034001BB10948802101F0E4FD2268094B9A4262
:1010440005D1094A1378B3FA83F35B09137010BD11
:10105400000001407C050020000C024080050020B7
:1010640084050020000C00400700002072B6FEE753
:101074000E480F4A08B54FF48273C0E900230023D9
:10108400C0E90233C0E90433C0E908334FF4007106
:10109400302283620A23C0E90612C36203F010FD02
:1010A40018B1BDE80840FFF7E1BF08BDC402002045
:1010B400003001400F48104A08B54FF48273C0E96C
:1010C4000023022100230122C0E90233C0E90412F3
:1010D400C0E908334FF4007C302283620A23C0E95C
:1010E40006C2C36203F0ECFC18B1BDE80840FFF788
:1010F400BDBF08BD1C030020003C00400E480F4A41
:1011040008B54FF48273C0E9002300234FF4007242
:10111400C0E90233C0E90433C0E90623C0E9083357
:1011240083620A23C36203F0CBFC18B1BDE8084014
:10113400FFF79CBF08BD00BF7403002000340140CA
:1011440010B504468CB01422002107A806F0C8FD8F
:101154002368394A934225D1384B394800210191FB
:101164005A6C42F480525A645A6C02F480520192CE
:10117400019A02911A6B42F001021A631B6B03F08D
:1011840001030293029B4FF0E00C0223CDE907C355
:101194004FF0030E0523CDE90AE307A901F052FC41
:1011A4000CB010BD274A934220D1244B0021039157
:1011B4001A6C42F400421A641A6C02F4004203925C
:1011C400039A04911A6B42F002021A631B6B03F038
:1011D400020304933820049B0223CDE9070303246C
:1011E4000623CDE90A43184807A9D7E7174A9342CB
:1011F400D6D1124B1648002105915A6C42F4005284
:101204005A645A6C02F400520592059A06911A6BBC
:1012140042F010021A631B6B03F010030693069B43
:101224004FF4E04202230321CDE907230523CDE94E
:101234000A1307A9B2E700BF00300140003802409A
:1012440000000240003C0040000402400034014021
:101254000010024082B00C4B002100915A6C42F401
:1012640080425A645A6C02F480420092009A0191BE
:101274001A6C42F080521A641B6C03F08053019381
:10128400019B02B0704700BF0038024070B588B0BF
:1012940000241D4B02945A6C1C4D42F001025A6406
:1012A4005B6C03F0010301A90293064603A8029BA9
:1012B40002F026FF02F014FF154B2B6040F2E733D7
:1012C400EB60144BB0FBF3F00138686028462C61E6
:1012D400AC60AC6104F06CF8044680B9284603F0B5
:1012E4001FFF044658B9192001F0A8F90F2E09D898
:1012F40022463146192001F06FF9074B1E60204643
:1013040008B070BD0124FAE700380240CC03002085
:101314000000014040420F0014000020FEE7FEE7F9
:10132400FEE7FEE7FEE7704770477047704701200D
:1013340001F070BC014801F0C7BA00BF8805002065
:10134400014801F0C1BA00BFE8050020014800F0DF
:10135400C4BF00BF38010020014803F020BF00BF14
:10136400CC030020014803F01ABF00BF140400207E
:10137400014803F014BF00BF5C040020014803F0DF
:101384000EBF00BFA4040020014804F08DBC00BFC0
:101394004806002008B54FF4806001F03BFC4FF490
:1013A400006001F037FC4FF4805001F033FC4FF43F
:1013B400005001F02FFC4FF4804001F02BFCBDE8FD
:1013C40008404FF4004001F025BC0000014803F040
:1013D400E6BE00BF34050020FFF7F8BFFFF7F6BFF5
:1013E400FFF7F4BF014803F0DABE00BFEC040020AD
:1013F400014801F069BA00BF80010020014802F0F1
:1014040021BA00BF701B0020B0F5806F08B50146FB
:101414000AD1154801F0EAFBB0FA80F252091348E8
:10142400042101F0E9FB08BDB0F5006FF1D0B0F57F
:10143400805FEED0B0F5804F07D0B0F5004F04D0F8
:10144400012804D0B0F5005FEDD1074800E008485A
:1014540001F0CCFBB0FA80F2BDE808400348520921
:10146400042101F0C9BB00BF00080240000402408F
:1014740000000240034AD2F8883043F47003C2F8F3
:101484008830704700ED00E07FB51022002102A8EB
:1014940006F026FC144847224FF080410023C0E99F
:1014A40000123122CDE90033C0E903238360836154
:1014B40003F07EFF08B1FFF7D9FD4FF480530A48CB
:1014C400029302A904F068F808B1FFF7CFFD0023E6
:1014D40005486946CDE9003304F072F908B1FFF715
:1014E400C5FD07B05DF804FB140400207FB510228D
:1014F400002102A806F0F4FB1448154941F61F42E6
:10150400C0E90012134A0023CDE90033C0E90323E4
:101514008360836103F04CFF08B1FFF7A7FD4FF42C
:1015240080530A48029302A904F036F808B1FFF781
:101534009DFD002305486946CDE9003304F040F9D8
:1015440008B1FFF793FD07B05DF804FBEC0400203D
:10155400000C0040A08601007FB50368B3F1804F02
:1015640016D1002203F50E330192196C41F00101EA
:1015740019641B6C03F0010301931C201146019BA9
:1015840001F02AF81C2007B05DF804EB01F056B80E
:10159400374A934211D1374B00220292196C41F021
:1015A400020119641B6C03F0020302931D2011460F
:1015B400029B01F011F81D20E5E72F4A934211D157
:1015C4002C4B00220392196C41F0040119641B6C2A
:1015D40003F0040303931E201146039B00F0FCFF59
:1015E4001E20D0E7254A934211D1224B00220492B7
:1015F400196C41F0080119641B6C03F0080304938F
:1016040032201146049B00F0E7FF3220BBE71C4A5E
:10161400934229D10022174B0592596C41F00201E3
:1016240059645B6C03F00203114605932B20059B60
:1016340000F0D2FF2B2001F001F8002211462C20EB
:1016440000F0CAFF2C2000F0F9FF002211462D20E3
:1016540000F0C2FF2D2000F0F1FF00222E201146E1
:1016640000F0BAFF2E208EE707B05DF804FB00BF40
:10167400000400400038024000080040000C004014
:101684000004014010B5044688B01422002103A8C8
:1016940006F026FB2368264A934217D100230093C1
:1016A400244B1A6B42F004021A631B6B03F004030D
:1016B40000934FF47070009B0223CDE903031E488E
:1016C400079303A901F0BEF908B010BD1B4A934269
:1016D40014D100230193174B19481A6B42F00802E6
:1016E4001A631B6B03F0080301934FF47041019BD1
:1016F4000223CDE90313079303A9E3E7114A9342B5
:10170400E2D1002302930B4B0F481A6B42F0020202
:101714001A631B6B03F002030293029B4FF44042D3
:101724000223CDE903230323079303A9CAE700BFD8
:101734000004004000380240000802400008004055
:10174400000C0240000401400004024010B58EB0B9
:101754001022002103A806F0C3FA00241C220DEB7A
:1017640002002146CDE9014406F0BAFA29482A4A82
:10177400846040F2CF23C0E900236423C0E903342A
:10178400846103F015FE08B1FFF770FC4FF4805339
:101794002048039303A903F0FFFE08B1FFF766FC9A
:1017A4001C4803F031FE08B1FFF760FC002419481F
:1017B40001A9CDE9014404F003F808B1FFF756FC90
:1017C400602314480994002207A9CDE907340B9437
:1017D40003F07CFE08B1FFF749FC0E48042207A978
:1017E40003F074FE08B1FFF741FC0A48082207A978
:1017F40003F06CFE08B1FFF739FC06480C2207A978
:1018040003F064FE08B1FFF731FC0248FFF73AFF2A
:101814000EB010BD5C0400200004004010B58EB072
:101824001022002103A806F05BFA00241C220DEB11
:1018340002002146CDE9014406F052FA29482A4A19
:10184400846040F2CF23C0E900236423C0E9033459
:10185400846103F0ADFD08B1FFF708FC4FF4805339
:101864002048039303A903F097FE08B1FFF7FEFB9A
:101874001C4803F0C9FD08B1FFF7F8FB0024194820
:1018840001A9CDE9014403F09BFF08B1FFF7EEFB8A
:10189400602314480994002207A9CDE907340B9466
:1018A40003F014FE08B1FFF7E1FB0E48042207A978
:1018B40003F00CFE08B1FFF7D9FB0A48082207A978
:1018C40003F004FE08B1FFF7D1FB06480C2207A978
:1018D40003F0FCFD08B1FFF7C9FB0248FFF7D2FE95
:1018E4000EB010BDA40400200008004010B596B04E
:1018F4001022002103A806F0F3F900241C2221463B
:101904000DEB0200CDE9014406F0EAF9202221465C
:101914000EA806F0E5F92C482C4A846040F2CF2347
:10192400C0E900236323C0E90334C0E9054403F09C
:101934003FFD08B1FFF79AFB4FF48053224803930D
:1019440003A903F029FE08B1FFF790FB1E4803F03A
:101954005BFD08B1FFF78AFB00241B4801A9CDE910
:10196400014403F02DFF08B1FFF780FB6023164804
:101974000D94042207A9CDE90734CDE90944CDE942
:101984000B4403F0A3FD08B1FFF770FB0E480822D7
:1019940007A903F09BFD08B1FFF768FB00234FF490
:1019A4000052094812930EA9CDE90E33CDE9103344
:1019B4001392159303F042FF08B1FFF757FB024857
:1019C400FFF760FE16B010BD34050020000401408E
:1019D40070B5434B434E1A798AB004461868009098
:1019E400D3F805008DF8042002905A7AD3F80A003F
:1019F4008DF80C2004909A7BD3F80F008DF81420F6
:101A04000690DA7C58698DF81C201B7E0890002211
:101A140020460D468DF8243001F0EEF84FF4805343
:101A240069460522304603F0A7F8294601222046DC
:101A340001F0E2F8012000F0ABFA2946204600222A
:101A440001F0DAF84FF4805302A90522304603F07E
:101A540093F829460122204601F0CEF8012000F037
:101A640097FA29462046002201F0C6F84FF4805325
:101A740004A90522304603F07FF8294601222046B6
:101A840001F0BAF8012000F083FA2946204600222A
:101A940001F0B2F84FF4805306A90522304603F052
:101AA4006BF829460122204601F0A6F8012000F037
:101AB4006FFA29462046002201F09EF84FF4805325
:101AC40008A90522304603F057F80122294620468A
:101AD40001F092F8012000F05BFA0AB070BD00BF7B
:101AE400387D00081C03002001480421FFF770BF63
:101AF4000010024001480821FFF76ABF00100240AD
:101B040001481021FFF764BF0010024038B5164C9D
:101B1400B4F91C30002B07D1BDE83840134801222A
:101B24004FF4004101F068B8114D10484FF0000225
:101B34004FF400410ADD01F05FF801220D4811461F
:101B440001F05AF8B4F91C302B6038BD01F054F898
:101B540008480022012101F04FF8B4F91C30002B91
:101B6400B8BF5B429BB2EFE73002002000000240A6
:101B74007C050020000C024038B5164CB4F91E3028
:101B8400002B06D1BDE8384013480122042101F09E
:101B940033B8124D10484FF000024FF004010ADD33
:101BA40001F02AF80C480122082101F025F8B4F9C3
:101BB4001E302B6038BD01F01FF8074800220821B1
:101BC40001F01AF8B4F91E30002BB8BF5B429BB287
:101BD400EFE700BF30020020000C02408005002027
:101BE40038B5164CB4F92030002B06D1BDE8384086
:101BF40013480122202100F0FFBF124D10484FF07E
:101C040000024FF020010ADD00F0F6FF0C4801222B
:101C1400402100F0F1FFB4F920302B6038BD00F012
:101C2400EBFF07480022402100F0E6FFB4F9203022
:101C3400002BB8BF5B429BB2EFE700BF300200202D
:101C4400000C0240840500200B480C4A08B54FF4F0
:101C5400E133C0E9002300230C22C0E90233C0E9C8
:101C640005230361C36103F09DFE18B1BDE808407C
:101C7400FFF7FCB908BD00BF48060020004400403F
:101C840070B5064688B01422002103A806F028F88F
:101C94003268314B9A425DD1002503F5FA33019540
:101CA4001A6C42F400321A641A6C02F40032019283
:101CB400019A02951A6B42F001021A631B6B03F03E
:101CC40001030293029B0C200223CDE903030324A6
:101CD4000723224803A9CDE9064300F0B3FE204CB4
:101CE400DFF888C04FF00063C4E900C320464FF416
:101CF4008063C4E90255C4E90435C4E90655C4E95E
:101D0400085500F0D1FC08B1FFF7B0F9154AB463E7
:101D1400A663154C4FF00063C4E90023402100235F
:101D24004FF480622046C4E90213C4E90423C4E9E1
:101D34000633C4E9083300F0B7FC08B1FFF796F99D
:101D44000022746326201146A66300F045FC262079
:101D540000F074FC08B070BD004400400000024074
:101D640088050020A0600240E80500208860024049
:101D7400064B834208D1064B01221A70054A137898
:101D8400B3FA83F35B091370704700BF4806002061
:101D94000800002027020020034B834202BF034BAC
:101DA40001221A70704700BF480600200600002078
:101DB4007FB54FF47A738DF80F0000930DF117027D
:101DC40001230DF10F01044802F084FF9DF8170070
:101DD40007B05DF804FB00BFC402002007B54FF450
:101DE4007A738DF8070001220DF10701044802F00F
:101DF400C3FE4FF44870FEF7E1FC03B05DF804FB4A
:101E0400C402002008B50A20FEF7D8FCBDE808404B
:101E1400FF20FFF7CDBF000013B50F4C8DF807006E
:101E240001221021204600F0E7FEC820FEF7C6FC80
:101E340020460022102100F0DFFE4FF47A730122C5
:101E44000DF10701054802F097FE40F2A460FEF789
:101E5400B5FC02B010BD00BF00000240C402002067
:101E640002480122102100F0C7BE00BF000002405A
:101E740008B51021034800F0B9FEB0FA80F040091B
:101E840008BD00BF0008024010B54FF4FA7000F01E
:101E94007FF80620FFF7C0FF5520FFF79FFFFFF7ED
:101EA400B1FF0446FFF7DCFFAA2C12D11520FFF77F
:101EB400B3FF0620FFF792FF1420FEF77FFCFFF725
:101EC400A1FF0446FFF7CCFF512C0CBF1420FA20CD
:101ED40010BDAA20FCE708B5FEF771FB143818BF43
:101EE400012008BDDFF834D00D480E490E4A002306
:101EF40002E0D458C4500433C4188C42F9D30B4ABA
:101F04000B4C002301E013600432A242FBD3FFF721
:101F1400B1FA05F0C1FEFEF7DBFF7047D8FF0120E0
:101F24000000002014010020D87D000814010020C6
:101F34009C220020FEE7000008B50B4B1A6842F40F
:101F440000721A601A6842F480621A601A6842F4D5
:101F540080721A60032000F02DFB0F20FFF796F922
:101F6400FFF778F9002008BD003C0240034A044B07
:101F740011681B780B441360704700BF8C06002067
:101F840010000020014B1868704700BF8C06002029
:101F940038B50446FFF7F6FF631C1CBF054B1B78DE
:101FA400054618BFE418FFF7EDFF431BA342FAD31D
:101FB40038BD00BF1000002038B50446002800F0EA
:101FC4009B80056C25B9FEF77DFB656484F83C5065
:101FD400236CDB0600F18E80236C23F4885323F0FA
:101FE400020343F002032364444B5A6822F4403250
:101FF4005A605A6861680A435A60236821695A68BA
:1020040022F480725A605A6842EA01225A605A687D
:10201400A16822F040725A605A680A435A609A686A
:10202400E16822F400629A609A680A439A6034492B
:10203400A26A8A4252D0996821F0706199609968C5
:102044000A439A609A68E16A22F040529A609A6858
:102054000A439A609A6822F002029A609A68217E82
:1020640042EA41029A6094F82020002A3ED05A683D
:10207400616A42F400625A605A6822F460425A600B
:102084005A68013942EA41325A60DA6AE16922F453
:102094007002DA62DA6A013942EA0152DA629A6853
:1020A40022F400729A609A6894F8301042EA41224D
:1020B4009A609A68616922F480629A609A68002042
:1020C40042EA81229A606064236C23F0030343F0A4
:1020D40001032364002384F83C3038BD9A6822F05D
:1020E40070629A609A6822F04052B2E75A6822F409
:1020F4000062C9E70120EDE70120EEE7002301407B
:102104000100000F73B513460022019290F83C20A1
:10211400012A054600F08C800122066880F83C20E4
:10212400B268D40754D5B268D00564D4B46814F046
:10213400010474D0286C20F4E06020F0010040F425
:10214400807028647268520541BF286C20F44050A6
:1021540040F4805028642A6CA86B12F480521CBF8F
:102164006A6C22F006026A640024334A85F83C4013
:10217400C263324A0264324AC2646FF0220232609D
:10218400726842F080627260B26842F48072B26037
:102194000A4606F14C0100F007FB2A4A2B685068F6
:1021A400294910F01F0032D18B4207D001F580710C
:1021B4008B4225D1526812F01F0F07D1986810F096
:1021C400405037D19A6842F080429A6002B070BDA4
:1021D400B26842F00102B2601C4A10681C4AB0FBAB
:1021E400F2F000EB40000190019A002A9BD0019A82
:1021F400013A0192F8E7B26822F48072B26095E77E
:1022040014498B42E2D1526812F0100FD5E78B4289
:1022140010D1986810F04050D4D02046D6E72B6CEB
:1022240043F010032B646B6C43F001036B64F4E71D
:102234000220CBE70020C9E711240008D1220008BE
:10224400FB23000800230140002001400C00002073
:1022540040420F000022014010B590F83C30012BA1
:10226400044630D00268012380F83C30936823F0A0
:1022740001039360936813F0010322D19168806B8A
:1022840021F48071916090F83520022A17D100F072
:10229400C5FA18B1236C43F04003236422685368E1
:1022A40023F080635360236C23F4885323F00103E9
:1022B40043F001032364002384F83C3010BD184626
:1022C400ECE70020F7E70220F8E7704708B5806BD9
:1022D400FFF7FBFF08BD70477047036870B51E68C1
:1022E4005D68B20704462BD5A80629D5226CD10611
:1022F4005EBF226C42F4007222649A6812F0405F5E
:1023040017D1227EAAB9DA6A12F4700F02D09A6841
:1023140052050ED45A6822F020025A60236C23F42A
:1023240080732364236CD8045EBF236C43F00103E1
:1023340023642046FEF730FA23686FF012021A6015
:10234400710733D52A0631D5236CDB065EBF236CB7
:1023540043F40053236423689A6812F4401F1ED187
:102364009A6B12F4401F02D09A68500517D45A6829
:10237400510514D49A6812F0405F10D1227E72B9CC
:102384005A6822F080025A60236C23F48053236439
:10239400236CDA055EBF236C43F0010323642046FB
:1023A40000F006F923686FF00C021A60F30710D5E9
:1023B40068060ED523681B68D9070AD5236C43F435
:1023C400803323642046FFF786FF23686FF0010201
:1023D4001A60B2060ED56B010CD5636C43F0020390
:1023E400636423686FF020051D602046FFF774FFC7
:1023F40023681D6070BD806B08B540230364436C83
:1024040043F004034364FFF767FF08BD836B1A6C52
:1024140012F0500F10B51A6C23D142F400721A64F2
:102424001A68916811F0405F17D1197EA9B9D16A71
:1024340011F4700F02D0916848050ED4516821F050
:10244400200151601A6C22F480721A641A6CD1044F
:102454005EBF1A6C42F001021A641846FEF79CF93A
:1024640010BDD20603D51846FFF736FFF8E79B6B7D
:10247400BDE81040DB6C1847F7B50023019390F8D2
:102484003C30012B69D0012380F83C300D6803688F
:102494008E68092DACB234D904EB4402DF681E3ACD
:1024A4004FF0070C0CFA02FC27EA0C07DF60DF6828
:1024B40006FA02F23A43DA604968062901EB81021E
:1024C4002FD8596B053A1F26964021EA0601596315
:1024D400596B04FA02F20A435A63304A93420AD10E
:1024E400122D3CD12E4B5A6822F400025A605A68CD
:1024F40042F480025A60002380F83C30184603B04E
:10250400F0BD1F6905EB45024FF0070C0CFA02FC05
:1025140027EA0C071F611F6906FA02F23A431A619F
:10252400CAE70C294FF01F010BD81E6B233A9140C8
:1025340026EA01011963196B04FA02F20A431A63C9
:10254400CBE7DE6A413A914026EA0101D962D96AB1
:1025540004FA02F20A43DA62BFE70220CFE7114B22
:102564009D4201D0112DC6D10D4B5A6822F4800230
:102574005A605A6842F400025A600A4B9D42BAD12A
:10258400094B0A4A1B68B3FBF2F30A225343019333
:10259400019B002BAFD0019B013BF8E700200140D9
:1025A40000230140120000100C00002040420F00E4
:1025B400704700000749CA6822F4E062030212046B
:1025C40003F4E063120C134343F0BF6343F400339A
:1025D400CB60704700ED00E0164B30B5DC68C4F307
:1025E4000224C4F10705231D042D28BF0425062B4E
:1025F4004FF0FF338CBF033C002403FA05F521EAB6
:102604000501A34022EA0302A140002841EA020393
:10261400ACBF00F16040084A4FEA0313B8BF00F0B2
:102624000F00DBB2AABF00F56140135480F80033F9
:1026340030BD00BF00ED00E014ED00E0002808DB31
:102644004209012300F01F0003FA00F0014B43F894
:102654002200704700E100E0BFF34F8F0549064BAD
:10266400CA6802F4E0621343CB60BFF34F8F00BF2C
:10267400FDE700BF00ED00E00400FA05036810B5B3
:10268400084C0246D9B210391820B1FBF0F0205C96
:10269400D06523F47F7020F003005F2988BF0430E5
:1026A400906510BD747D000870B50446FFF76AFCA0
:1026B4000546002C73D0022384F8353022680023A9
:1026C40084F83430136823F00103136021680B6825
:1026D400D8072FD40B68334DA0691D40D4E90123DA
:1026E4001343E26813432269134362691343E269A3
:1026F40003431343226A1343626A042A43EA050329
:1027040002BFD4E90B5635432B430B604B69042AB3
:1027140023F0070343EA020333D1A26AE56A1343B1
:102724007DB390B9012A21D032F0020229D1EA0105
:1027340027D51EE0FFF726FC401B0528C6D9202319
:102744006365032084F8350070BDB0F5005F14D1D3
:10275400032A16D801A050F822F000BF77270008FA
:10276400332700087727000871270008B5F1C07FD8
:1027740007D1402363650120E4E7022AF9D9032A3B
:10278400D5D04B612046FFF779FFE26D3F2393409C
:10279400836000200123606584F83530D4E701208C
:1027A400D2E700BF3F8010F070B590F83440866DDA
:1027B400012C31D0012480F8344090F83540012CAC
:1027C4004FF000054FF0020424D180F8354004682E
:1027D4004565256825F48025256063608368402B62
:1027E4000EBFA260A160E260C26D08BFE1603F233A
:1027F4009340B360236843F016032360036C1BB15A
:10280400236843F008032360236843F00103236033
:10281400002070BD80F834500220FAE770B50446F9
:10282400866DFFF7AFFB94F83530022B054606D0D2
:1028340080236365002384F83430012070BD23684D
:102844001A6822F016021A605A6922F080025A614C
:10285400226C0AB9A26C1AB11A6822F008021A6032
:102864001A6822F001021A6023681B6813F001033E
:102874000AD1E16D3F228A40B260012284F83520FA
:1028840084F834301846D9E7FFF77CFB401B052851
:10289400EAD9202363650320002384F8350084F8F3
:1028A4003430CBE790F83530022B03D080234365D6
:1028B400012070470268052380F83530136823F03F
:1028C4000103136000207047F7B5002301935C4BAC
:1028D400856D1F68C36D2E6808229A4032420446F3
:1028E4000CD001680868400708D5086820F0040087
:1028F4000860AA60626D42F00102626501229A409A
:10290400324208D021684969090641BFAA60626D54
:1029140042F00202626504229A40324208D02168E1
:102924000968880741BFAA60626D42F004026265CB
:1029340010229A40324210D02368196809070CD536
:10294400AA601A68500337D51B68190301D4236C95
:1029540000E0A36C0BB120469847E16D20228A4029
:1029640032423AD023681868C60636D5AA6094F86D
:102974003520052A1A6827D122F016021A605A69EE
:1029840022F080025A61226C0AB9A26C1AB11A6848
:1029940022F008021A603F238B40AB60012384F8C5
:1029A4003530002384F83430236D002B45D0204685
:1029B40003B0BDE8F04018471A68D2055EBF1A6834
:1029C40022F008021A60C2E7500327D51B681903D6
:1029D40031D4636C0BB120469847636D6BB3636D60
:1029E400DA0719D522684FF41653B7FBF3F705231A
:1029F40084F83530136823F001031360019B01331D
:102A0400BB42019302D81368DB07F7D4012384F88F
:102A14003530002384F83430E36CC6E71A6812F4C6
:102A2400807208D1196821F010011960012384F81B
:102A3400353084F83420E36BCCE703B0F0BD00BF3D
:102A44000C0000202DE9F74FDFF89C91644A002325
:102A54000D6801249C4004EA050CAC4340F0AD80B1
:102A64004D6805F003044FEA43080326671E06FA7F
:102A740008F6012F6FEA060634D8876807EA060EBF
:102A8400CF6807FA08F747EA0E078760476827EA1E
:102A94000C0EC5F300179F4047EA0E074760C7684E
:102AA40007EA060E8F6807FA08F747EA0E07022CB2
:102AB400C76019D14FEAD30A00EB8A0A03F0070B67
:102AC400DAF820704FEA8B0B4FF00F0E0EFA0BFE64
:102AD40027EA0E0E0F6907FA0BF747EA0E07CAF842
:102AE400207001E0032CDAD1076804FA08F43E40B0
:102AF400264315F4403F06605FD04FF0000ACDF83E
:102B040004A0D9F84460374C46F48046C9F84460C0
:102B1400D9F8446006F480460196019E23F003062A
:102B240006F1804606F59C3603F0030ED6F80880BD
:102B34004FEA8E0E0F2707FA0EF7A04228EA07077E
:102B440042D004F58064A04240D004F58064A042E1
:102B54003ED004F58064A0423CD004F58064A042D9
:102B64003AD004F58064A04238D004F58064A042D1
:102B74000CBF0624072404FA0EF43C43B4609468A2
:102B84006FEA0C06EF0254BF34404CEA040494602C
:102B9400D468AF0254BF34404CEA0404D46054688F
:102BA400AF0354BF34404CEA040454601468ED038A
:102BB40054BF34404CEA040414600133102B7FF4F6
:102BC40047AF03B0BDE8F08F5446D4E70124D2E701
:102BD4000224D0E70324CEE70424CCE70524CAE783
:102BE400003C0140000002400038024003691942E1
:102BF40014BF0120002070470AB1816170470904A5
:102C0400FBE7436901EA030221EA030141EA0241C5
:102C140081617047044A5169014208B502D050618C
:102C2400FEF7F2FB08BD00BF003C014001684B69A0
:102C340013F480634FF0000210D06FF480634B6193
:102C44002023026380F83D3080F83E20036C80F836
:102C54003C2043F004030364012070471846704786
:102C64002DE9F84606460F4691461D464FEA114A9D
:102C74003368BAF1010F0CBF5C699C6927EA04044C
:102C8400A4B2B4FA84F46409A14501D0002017E089
:102C94006A1CEED0FFF776F9089BC01AA84201D847
:102CA400002DE5D100232022336386F83D2086F8E9
:102CB4003E30326C86F83C3042F02002326401200F
:102CC400BDE8F8862DE9F04104460F4616469846BD
:102CD4002568686927EA000080B2B8B16B695A05B3
:102CE40016D52B6843F400732B606FF480636B611B
:102CF40020220023236384F83D2084F83E30226C94
:102D040042F00402226484F83C300120BDE8F081E2
:102D1400731CDED0FFF736F9A0EB0800B04201D8EF
:102D2400002ED5D100232022236384F83D2084F88B
:102D34003E30226C42F02002E4E770B504460D46B2
:102D4400164621684B6913F0400301D0002010E0BF
:102D54004A69D2060ED56FF010024A61202223631D
:102D640084F83D2084F83E30226C226484F83C30A0
:102D7400012070BDFFF706F9801BA84201D8002D81
:102D8400DFD100232022236384F83D2084F83E30E1
:102D9400226C42F02002E8E770B504460D46164660
:102DA40023685B695B0701D5002070BD2046FFF7EF
:102DB4003DFFA8B96A1CF3D0FFF7E4F8801BA842D2
:102DC40001D8002DECD100232022236384F83D2078
:102DD40084F83E30226C84F83C3042F020022264B5
:102DE4000120E2E770B504460D46164623685B6988
:102DF4001B0601D5002070BD2046FFF717FFA8B9B8
:102E04006A1CF3D0FFF7BEF8801BA84201D8002D3E
:102E1400ECD100232022236384F83D2084F83E3043
:102E2400226C84F83C3042F0200222640120E2E764
:102E34002DE9F0431546026885B0DDE90C78994622
:102E4400136843F4807313600E463B46CDF800804C
:102E540000224FF001110446FFF702FF236838B146
:102E64001B68DB0502D54FF40073236403200AE0DA
:102E740006F0FE061E61194943463A462046FFF70E
:102E840021FF18B1012005B0BDE8F0832368039049
:102E94005A6903929B690393424639462046039B31
:102EA400FFF7A0FF40B1236C042B01BF2268136815
:102EB40043F400731360E5E7B9F1010F236802D10D
:102EC400EDB21D61DFE72A0A1A61394642462046FF
:102ED400FFF788FF0028E6D12368F1E7020001002C
:102EE4002DE9FF479A46036815461A6842F4806242
:102EF4001A601A68DDE90C7842F480721A600E4692
:102F04003B46CDF8008000224FF001110446FFF744
:102F1400A7FE236848B11B68DB0502D54FF4007394
:102F24002364032004B0BDE8F0875FFA86F906F055
:102F3400FE061E612A4943463A462046FFF7C2FE72
:102F440008B10120EEE7236803905A6903929B6954
:102F54000393424639462046039BFFF743FF40B1A3
:102F6400236C042B01BF2268136843F400731360BD
:102F7400E7E7BAF1010F23681AD1EDB21D614246A9
:102F840039462046FFF72EFF0028E9D1226813684E
:102F940043F4807313604FF001110246CDF80080B2
:102FA4003B462046FFF75CFE226860B11368B3E736
:102FB4002A0A1A61394642462046FFF713FF0028C1
:102FC400CED12368D9E749F001031361044943468C
:102FD4003A462046FFF776FE003818BF0120A1E7E5
:102FE4000200010070B5044608B9012070BD90F8D4
:102FF4003D3003F0FF021BB980F83C20FDF7E0FEF2
:10300400242384F83D3023681A6822F001021A60F0
:103014001A6842F400421A601A6822F400421A60E4
:1030240001F04EF83F4B65689D4294BF3E4B3F4BC9
:1030340098428CBF00230123002BD6D12268394E3D
:1030440053683B49B0FBF1F123F03F030B43B54216
:10305400536088BF4FF49676136A88BF714323F098
:103064003F0384BF4FF47A76B1FBF6F10131194383
:103074001162D169431E2B4821F44F41854221F04E
:10308400FF0132D86D0040F6FC70B3FBF5F3013359
:10309400034242D0C3F30B030B43D361D4E907309B
:1030A4001168034321F0C0010B4313609168D4E914
:1030B400030321F40341034321F0FF010B43936015
:1030C400D4E90530D168034321F0FF010B43D360F9
:1030D400136843F00103136000202023206484F864
:1030E4003D30206384F83E0080E7A06850B905EBCA
:1030F4004505B3FBF5F30133C3F30B037BB143F491
:103104000043C9E719204543B3FBF5F30133C3F387
:103114000B0323B143F44043BEE70423BCE701237C
:10312400BAE700BFA08601007F841E00FF083D00AF
:1031340040420F002DE9F743044699460C9E0F4682
:103144009046FEF71FFF94F83D30202B054603D030
:10315400022003B0BDE8F08300903C49192301220A
:103164002046FFF77DFD0028F2D194F83C30012B76
:10317400EED02068012384F83C300368D9075EBF91
:10318400036843F001030360036823F400630360EE
:10319400212384F83D30402384F83E300023236407
:1031A4000A9B6362BDF82C306385638D2385284BAD
:1031B400E362CDE900654B46424639462046FFF7B7
:1031C40037FE00282AD00120C3E7FFF70BFE40B1E9
:1031D400236C042B01BF2268136843F4007313604B
:1031E400F1E7636A27681A4612F8011B39616262C3
:1031F400628D218D013A92B262857A69481E80B24D
:10320400520720850AD548B15A783A61023363627D
:10321400638D013B02399BB221856385238D2A4648
:1032240031462046002BD0D1FFF7B6FD0028CFD180
:103234002268136843F400731360202384F83D303C
:1032440084F83C0084F83E0083E700BF02001000CD
:103254000000FFFF2DE9F043044687B09946109F14
:103264000D469046FEF78EFE94F83D30202B064620
:1032740004D00225284607B0BDE8F08300907649C3
:10328400192301222046FFF7EBFC0028F1D194F822
:103294003C30012BEDD02068012384F83C300368D6
:1032A400DB075EBF036843F001030360036823F494
:1032B40000630360222384F83D30402384F83E30C9
:1032C400002323640E9B6362BDF83C306385638DE9
:1032D4002385624BE3622946CDE900764B4642469C
:1032E4002046FFF7FDFD054608B10125C2E7228D02
:1032F4002368B2B902905A6902929A690292029AB8
:103304001A6842F400721A60DFF85481238D002B8E
:103314002CD1202284F83D2084F83C3084F83E30BF
:10332400A8E7012A0AD11A6822F480621A6003907D
:103334005A6903929A690392039AE1E7022A0ED129
:103344001A6822F480621A601A6842F400621A60F1
:1033540004905A6904929B690493049BD4E70590F2
:103364005A6905929B690593059BCDE7032B56D8B3
:10337400012B15D1324639462046FFF7DEFC0028E2
:10338400B3D123681A69636A1A70636A013363628A
:10339400238D013B2385638D013B9BB26385B5E798
:1033A400022B00963B464FF000024146204619D1BD
:1033B400FFF756FC002898D123681A6842F400727B
:1033C4001A601A69636A1A70626A531C6362238DF5
:1033D400013B2385638D013B9BB2638523681B6995
:1033E4005370D2E7FFF73CFC00287FF47EAF2368DC
:1033F4001A6822F480621A601A69636A1A70636A2E
:10340400009601336362238D013B2385638D013B69
:103414009BB2638502463B4641462046C8E7324696
:1034240039462046FFF789FC00287FF45EAF236805
:103434001A69636A1A70626A531C6362238D013BC2
:103444002385638D013B9BB26385236859694907D2
:103454007FF55CAFC3E700BF020010000000FFFF70
:1034640004000100F0B504468BB060B390F8BD349D
:10347400056803F0FF021BB980F8BC2404F090FA3D
:10348400032384F8BD34EB6B254613F4807355F89D
:10349400100B08BF236102F099FE0FCD6E460FC6D4
:1034A4000FCD0FC695E8030086E803002546271DC7
:1034B40097E80E0055F8100B02F0D2FD064620B135
:1034C400022384F8BD34012554E00146206802F04B
:1034D40083FE3046D4F804C024264FF0010E014682
:1034E400C2B2944500F101001CD8002324261946D9
:1034F400D8B2844503F1010322D80FCD6E460FC61E
:103504000FCD0FC695E8030086E8030097E80E0088
:10351400206802F0E3FE01230546F0B1022284F89C
:10352400BD24D0E706FB0243C3E9121183F83DE052
:1035340083F83C20A3F8442083F840105965CFE772
:1035440006FB0042C2E9A21182F87D1282F87C02D5
:1035540082F88012C2F89412CAE784F8380084F81A
:10356400BD34636A012B02D1204600F0F3FC2068CD
:1035740003F05AFA28460BB0F0BD10B504460068B3
:1035840094F8BC34012B15D0012384F8BC34A36A0D
:10359400012B06D1A369012B1EBF836B43F4803337
:1035A400836302F00DFE206803F030FA002084F8F3
:1035B400BC0410BD0220FCE710B590F8BC24012A1D
:1035C40004460BD0012280F8BC2480F8381000682F
:1035D40003F00CFA002084F8BC0410BD0220FCE7C0
:1035E40070B501F00F0606EBC60411F0800F054616
:1035F4004FEA84044FF024001FD000FB065004F16E
:103604003C010124294480F83D40CA604A780E7088
:103614000B7102B10E81022B04BF00234B7195F88C
:10362400BC34012B12D00123286885F8BC3402F085
:1036340016FF002085F8BC0470BD00FB065004F59D
:103644001F710024294480F87D42DEE70220F3E75D
:1036540010B5044601F00F0000EBC00311F0800F19
:103664004FEA83034FF0240216D002FB004203F119
:103674003C010123214482F83D30087094F8BC34A5
:10368400012B12D00123206884F8BC3402F026FFF9
:10369400002084F8BC0410BD02FB004203F51F7136
:1036A4000023214482F87D32E7E70220F3E738B5AE
:1036B40001F00F05242404FB050104FB050401F5B6
:1036C4001F71C4F894320023C4F88C22C4F89C32CD
:1036D40084F87D3284F87C5203690068012B08BFAA
:1036E400C4F89022DAB21DB902F04EFF002038BDB2
:1036F40003F01CF8FAE701F00F01242303FB010097
:10370400D0F89C02704738B501F00F05242404FB5F
:10371400050104FB05043C3163650023E3650123D3
:10372400E26484F83D3084F83C5003690068012B5E
:1037340008BF2265DAB21DB902F026FF002038BDA9
:1037440002F0F4FFFAE738B5436801F00F059D4233
:1037540004462CD811F0800F4FF024001ED000FB3B
:10376400054200FB054101233C3182F83D30012331
:103774008B700D7094F8BC249A421AD0206884F897
:10378400BC3403F0DFF82DB9217C206804F2C44274
:1037940003F09CF9002084F8BC0438BD00FB01430D
:1037A4001A4603F51F71002382F87D32DFE70120FA
:1037B400F3E70220F1E738B5436801F00F029A42BB
:1037C40004462AD802EBC20311F0800F4FEA8303A8
:1037D4004FF0240018D000FB024003F13C01012308
:1037E400214480F83D3000258D700A7094F8BC3473
:1037F400012B14D00123206884F8BC3403F0CDF8E5
:1038040084F8BC54284638BD00FB024003F51F7100
:103814000023214480F87D32E5E70120F3E702200C
:10382400F1E701F00F0303EBC3030A064FEA830336
:103834004CBF03F13C0103F51F710144006802F021
:103844001FBF00002DE9F04F066889B004463046DA
:1038540003F027F90390002840F07081206803F0FA
:10386400F1F8002800F06A81D6F808382068C3F31C
:103874000D23C4F8FC3403F0E5F8810748BF22683F
:10388400206842BF536903F00203536103F0DAF87E
:10389400C20606F500652CD52268936923F010034F
:1038A4009361D6F82080C8F34343022B08F00F0736
:1038B40040F0478147F6F07318EA030F14D024232D
:1038C40003FB0747C8F30A19D7F88C124A46304657
:1038D40003F018F8D7F88C324B44C7F88C32D7F879
:1038E4009C324B44C7F89C322268936943F010031E
:1038F4009361206803F0A6F8030300F13481206883
:1039040003F0A0F847030CD5206803F0A7F8274676
:10391400049006F5106A4FF00009049B002B40F058
:10392400EA81206803F08EF8002813DA6B6823F02C
:1039340001036B6094F8F434012B40F0858200217C
:1039440084F8F414204604F01BF92268536903F048
:1039540000435361206803F075F800050AD5AB688D
:10396400D90702D5204604F099F82268536903F474
:1039740000635361206803F065F8020114D52368DD
:103984005A6902F000625A6194F8F424002A40F063
:103994005F82012184F8F4145B6DC3F38303C4F8DC
:1039A400F834204604F0ECF8206803F04BF8C30424
:1039B40033D56B68206823F001036B60102102F09B
:1039C4003BFC06F510634FF67F3162680398824230
:1039D40000F24682EB6943F00113EB61236B002B89
:1039E40000F05682D5F8843043F00B03C5F88430D8
:1039F4006B6C43F00B036B64D6F80038217C2068B1
:103A040023F4FE63C6F8003804F2C44203F05EF8FF
:103A14002268536903F480535361206803F012F859
:103A2400870416D5206803F040F8206802F00CFDE6
:103A3400E060276800F03EFB227B0146384602F036
:103A44004FFB204604F017F82268536903F400532F
:103A54005361206802F0F6FF000707D5204604F002
:103A640006F82268536903F008035361206802F0E2
:103A7400E9FF010600F11782206802F0E3FFC202A9
:103A84000CD5A04606F5126901276368BB4200F213
:103A940023822268536903F480135361206802F07F
:103AA400D1FF83022DD5D4F804E0234606F5326015
:103AB40001218E4520D993F8A4C20268BCF1010FFC
:103AC40040F02082002A80F21D82D4F8FC7402F4B3
:103AD400803207F00107BA4240F0148283F8A3C28F
:103AE400B26942F08002B2617269170600F10A827B
:103AF4006B6843F400736B602268536903F400132A
:103B04005361206802F09EFF410007D5204603F070
:103B1400E9FF2268536903F080435361206802F08F
:103B240091FF42070AD523685D686B0702D52046DA
:103B340003F0DCFF226853682B43536009B0BDE8EF
:103B4400F08F062B7FF4D0AE082204F2C441304635
:103B540002F0D8FE242303FB0747C8F30A18D7F85A
:103B64009C324344BEE6206802F070FF06F53068DC
:103B74000490A2460027049B002B3FF4C0AE049B94
:103B8400D80776D55FFA87FB2068594602F06EFFA6
:103B940010F0010F81461CD0206821690123C8F868
:103BA400083000F5306303EB47130129D0F840C017
:103BB4009A6840F08B80110707D5A7498C4508D92E
:103BC400100406D54FF4004202E091065AD5202293
:103BD4009A6019F0080F21D00823C8F80830236828
:103BE4009D481A6C03F5306303EB471382429968CE
:103BF40004D9090444BF4FF400419960204605925A
:103C040003F01EFF944B059A9A4207D921690129B2
:103C140004D1206804F2C44202F058FF19F0100FD6
:103C24001CBF1023C8F8083019F0020F14D07369B0
:103C34001A0642BF6B6843F480636B609AF87F3264
:103C4400012B06D100238AF87F325946204603F01F
:103C540041FF0223C8F8083019F0200F1CBF2023AD
:103C6400C8F8083019F4005F1CBF4FF40053C8F8BB
:103C74000830049B5B080137049308F120080AF11B
:103C8400240A78E712F0280FA3D173498C4501D98F
:103C9400120497D41A69DAF89832C2F312029B1A02
:103CA400CAF89C326FB9D4F894222AB904F2C442F7
:103CB400012102F00BFF04E0D4F88C221344C4F871
:103CC4008C325946204603F0C1FE82E763498C4595
:103CD40007D111043FF576AF9006F2D520229A6001
:103CE400EFE7002FEDD1D4F89432002BE9D104F2A0
:103CF400C4423946DDE7049BDB0740F19C805FFA50
:103D040089FB2068594602F0BAFE10F0010F804684
:103D140020D001216B6B09F00F0201FA02F223EAB1
:103D240002036B630B46CAF80810216999420DD14E
:103D3400D7E912231344FB64B9F1000F06D1636D74
:103D440023B9206804F2C44202F0C0FE594620465A
:103D540003F085FE18F0080F1CBF0823CAF80830CA
:103D640018F0100F1CBF1023CAF8083018F0400FC9
:103D74001CBF4023CAF8083018F0020F12D049467D
:103D8400304602F059FA97F83F30012B07D14FF033
:103D9400000387F83F305946204603F09FFE022374
:103DA400CAF8083018F0800F45D0FA6D7B6D9A423E
:103DB40041D89B1ABA6C21680591934228BF1346D7
:103DC40003339B08069301F5106303EB4913079330
:103DD400079B06989969FA6D7B6D89B2814228D355
:103DE4009A420CD3059B09F00F01D3F83428012023
:103DF40000FA01F122EA0102C3F834281BE0A3EB24
:103E04000208BB6C0598984528BF984608F103033F
:103E14009B080693237C0093F96C1FFA88F35A4697
:103E240002F070FCFB6C4344FB64FB6D4344FB6594
:103E3400CEE79A42D6D2049B5B0809F101090493A8
:103E440024370AF1200A68E5204603F03FFE7CE5AA
:103E5400204603F023FEA7E50A30544F0A31544F9D
:103E640099601A6822F400121A60C3F80812D3F891
:103E7400002222F40012C3F80022D3F8002242F0F8
:103E84000062C3F80022039A0132039220339CE5B6
:103E94006B6943F4005343F02B036B612B6943F0CC
:103EA4000B032B61A8E5B36923F08003B3610127F9
:103EB40004F27F284FF024096368BB427FF6DCAD2F
:103EC40009FB07F318F80330012B03D1F9B220469C
:103ED400FFF7A7FC0137EFE798F86430D9F8002022
:103EE400012B09D1002A07DA67F07F0188F86330D3
:103EF400C9B22046FFF795FC013708F1240809F1FF
:103F04002009C2E5013124332030D2E5006870B5C0
:103F14001204446A19B922438262002070BD836A84
:103F24004D1E04EB134400235E1CDBB29D4205D8F6
:103F34003F3100EB810022434260EEE7403300EB67
:103F440083035B6804EB13443346EDE70368002006
:103F5400596270470268002180F8F4140123C0F804
:103F64000035936943F000639361536D43F08053CC
:103F740043F0030353650846704700002DE9F04100
:103F84000D46044610B90120BDE8F081444B1A687F
:103F940002F00F028A4228D3226897072DD4D00753
:103FA40041D43F4B1A6802F00F02AA4266D8226835
:103FB40051076CD4130707D53A4A2169936823F44F
:103FC400604343EAC103936000F0C0FA354B364ABC
:103FD4009B68C3F30313D35CD840344B1860344B51
:103FE4001868FDF753F90020CEE7CAB21A701B68AF
:103FF40003F00F038B42C6D1CEE72A4B12F0040F15
:104004001EBF996841F4E0519960160742BF996850
:1040140041F4604199602349A0688B6823F0F00360
:1040240003438B60BBE762681E4B012A1CD11B68EB
:1040340013F4003FA7D01B4EB36823F003031343CC
:10404400B360FDF79FFF41F288380746B3686268A2
:1040540003F00C03B3EB820FA3D0FDF793FFC01B57
:104064004045F3D903208FE7911E01291B6802D82C
:1040740013F0007FDEE713F0020FDBE7EAB21A70F9
:104084001B6803F00F03AB427FF47DAF8FE7054954
:10409400E0688B6823F4E05303438B608AE700BF36
:1040A400003C0240003802405C7D00080C00002007
:1040B40014000020014B1868704700BF0C0000205A
:1040C400044B054A9B68C3F38223D35C034A1068FC
:1040D400D8407047003802406C7D00080C00002076
:1040E400044B054A9B68C3F34233D35C034A10680C
:1040F400D8407047003802406C7D00080C00002056
:104104000F2303600B4B9A6802F0030242609A6823
:1041140002F0F00282609A6802F4E052C2609B6886
:10412400DB0803F4E0530361034B1B6803F00F0344
:104134000B60704700380240003C024003682DE9E0
:10414400F74313F0010604460BD0AB49866BD1F854
:104154008C2022F0C0623243B6FA86F6C1F88C2075
:1041640076099A070BD5A448E16BD0F88C2022F08D
:10417400C0520A430029C0F88C2008BF012613F05E
:10418400040512D09C49256BD1F88C20B5F5801F0D
:1041940022F4401242EA050218BFB5FA85F5C1F8C7
:1041A4008C2012BF6D09002501261F070FD59248E8
:1041B400616BD0F88C2022F440020A43B1F5800FE1
:1041C400C0F88C2000F00A81002908BF0125980658
:1041D40033D500230193884B884F1A6C42F08052E8
:1041E4001A641B6C03F080530193019B3B6843F4F6
:1041F40080733B60FDF7C6FE80463B68D90540F1FD
:10420400EF807D4F3B6F13F4407340F0FD80236CCF
:1042140003F44072B2F5407F774A40F01A81916806
:1042240023F0704021F4F81120F4407001439160B0
:10423400116FC3F30B030B4313672368D80642BF04
:104244006F4B94F85820C3F8E0212368190608D569
:104254006949E06CD1F8942022F440020243C1F889
:1042640094205A0608D56449A06CD1F8942022F011
:1042740080620243C1F89420DF050CD55E48616D6D
:10428400D0F8942022F000620A43B1F1006FC0F824
:10429400942008BF0125980508D55749606CD1F8CA
:1042A400942022F080520243C1F89420590500F171
:1042B400D480012E40F0DF80524B4F4E00229A668C
:1042C400FDF760FE074633681A0100F12881226871
:1042D400D30701D5A36B1BB1970714D5E36B93B92F
:1042E400D6F88430D6F8841003F4403301F07061BA
:1042F4000B4361680B43A16843EA8113616943EA94
:104304000173C6F88430560703D5236BB3F5801FB9
:1043140005D0100720D5636BB3F5800F1CD1364947
:10432400D1F88430D1F8840003F4403300F0E04045
:10433400034360680343A06843EA8013206943EAA7
:104344000063C1F88430D1F88C00A36A20F01F0008
:10435400013B0343C1F88C3051051BD5236DB3F1E8
:10436400005F17D124486668D0F88410D0F88430F0
:1043740003F0E0433343A668C1F30141013143EA4A
:10438400861343EA4163E1684908013943EA01437A
:10439400C0F88430120511D52369A2681B0643EACC
:1043A400821362681343626943EA0273E268520843
:1043B400013A43EA0243104AC2F88430114B0E4FCB
:1043C40001229A66FDF7DEFD06463B681B0156D4C2
:1043D400FDF7D8FD801B0228F7D908E00126F6E690
:1043E400FDF7D0FDA0EB080002287FF606AF0320FE
:1043F40003B0BDE8F08300BF003802400070004005
:104404000010474200004742226C02F440729A4274
:104414003FF4FDAE3B6F4B4A0121C2F8401E23F42A
:1044240040730021C2F8401E3B673B6FDA077FF5FB
:10443400EEAEFDF7A7FD41F2883980463B6F9B073E
:104444003FF5E5AEFDF79EFDA0EB08004845F5D924
:10445400CDE7916821F4F811E9E63B48216DD0F8E5
:10446400942022F000520A43B1F1005FC0F8942076
:104474007FF41FAF20E7B3F5006F3FF41DAF012DAC
:104484004BD1304B304D00221A67FDF77BFD0646B9
:104494002B689F004AD42268500701D5236B1BB1B7
:1044A400110719D5636BBBB9D5F88830A16903F43A
:1044B40040330B43E16943EA8113616A43EA0163D0
:1044C400C5F88830D5F88C30E16A23F4F853013903
:1044D40043EA0123C5F88C30D20514D5636DB3F1DA
:1044E400006F10D11849A269D1F8883003F07063C5
:1044F4001343E26943EA8213226A5208013A43EA07
:104504000243C1F888300F4B0F4D01221A67FDF7A3
:1045140039FD04462B689B000ED5002068E7FDF7A3
:1045240031FDC01B02287FF6CEAE60E7FDF72AFD01
:10453400801B0228ACD95AE7FDF724FD001B022892
:10454400E8D954E70000474200380240204908B542
:104554008B6803F00C03082B07D00C2B20D01D48CC
:104564001D4A042B08BF104608BD4A684B684968B9
:1045740013F4800314BF18481648C1F3881118BFF8
:10458400002302F03F02A1FB0001FBF741FE104BA8
:104594005B68C3F3014301335B00B0FBF3F0E3E773
:1045A4004A684B68496813F4800314BF0A480948F1
:1045B400C1F3881118BF002302F03F02A1FB0001E0
:1045C400FBF726FE024B5B68C3F30273E5E700BF0B
:1045D400003802400024F400001BB7002DE9F34129
:1045E4000446002830D00368DF0710D423689E07F0
:1045F40063D423681A0700F1AD8023685B0700F1D8
:10460400CD80A069002840F03581002034E0964B2D
:104614009A6802F00C02042A0FD09A6802F00C0285
:10462400082A02D15A68550207D49A6802F00C028B
:104634000C2A0BD15B68580208D58B4B1B68990375
:10464400D4D56368002BD1D1012015E06368864D71
:10465400B3F5803F13D12B6843F480332B60FDF70F
:1046640091FC814E054633689A03BFD4FDF78AFC5A
:10467400401B6428F7D9032002B0BDE8F081B3F5EC
:10468400A02F04D12B6843F480232B60E3E72A682E
:1046940022F480322A602A6822F480222A60002BC5
:1046A400DDD1FDF76FFC06462B689B039ED5FDF715
:1046B40069FC801B6428F7D9DDE76B4B9A6812F01C
:1046C4000C0F0FD09A6802F00C02082A02D15A6823
:1046D400570207D59A6802F00C020C2A11D15B68C4
:1046E4005E020ED4604A13689D0702D5E368012B6D
:1046F400AAD11368216923F0F80343EAC1031360C4
:1047040077E7E268594BB2B101221A60FDF73AFC2F
:10471400554D06462B68980707D52B68226923F068
:10472400F80343EAC2032B6063E7FDF72BFC801B0D
:104734000228EFD99FE71A60FDF724FC4A4E05468C
:10474400336899077FF555AFFDF71CFC401B022821
:10475400F6D990E76269454B82B10122C3F8802EF5
:10476400FDF710FC404E0546736F9F073FF545AFBC
:10477400FDF708FC401B0228F6D97CE7C3F8802E1D
:10478400FDF700FC384E0546736F98077FF535AF8B
:10479400FDF7F8FB401B0228F6D96CE7324B1A6C84
:1047A40012F0805228D101921A6C42F080521A649D
:1047B4001B6C03F080530193019B01272C4D2B6844
:1047C400D9051BD5A368284D012B27D12B6F43F0A6
:1047D40001032B67FDF7D6FB234E054641F28838CB
:1047E400336F9B0739D5002F3FF40BAF1E4A136C70
:1047F40023F08053136404E70027DFE72B6843F4B6
:1048040080732B60FDF7BEFB06462B68DA05D9D40E
:10481400FDF7B8FB801B0228F7D92CE7052B04D140
:104824002B6F43F004032B67D0E72A6F22F00102B9
:104834002A672A6F22F004022A67002BCAD1FDF7E7
:10484400A1FB41F2883806462B6F9807CBD5FDF7BC
:1048540099FB801B4045F7D90DE7FDF793FB401BFF
:104864004045BDD907E700BF003802400000474279
:10487400007000403B4DAB6803F00C03082B40D0A4
:10488400394B002202281A662ED1FDF77BFB06461F
:104894002B68990122D4D4E907321343626A43EAAC
:1048A4008213E26A43EA0263226B43EA0273A26A56
:1048B4005208013A43EA02436B602B4B294D012213
:1048C4001A66FDF75FFB04462B689A013FF59DAE1F
:1048D400FDF758FB001B0228F6D9CCE6FDF752FB86
:1048E400801B0228D4D9C6E6FDF74CFB04462B688E
:1048F4009B017FF58AAEFDF745FB001B0228F6D924
:10490400B9E601283FF4B8AE6B68E26903F48001AC
:1049140091427FF499AE216A03F03F028A427FF408
:1049240093AE616A47F6C0721A40B2EB811F7FF4FE
:104934008BAEA26A520803F44031013AB1EB024F44
:104944007FF482AEE16A03F07062B2EB016F7FF430
:104954007BAE226B03F0E043B3EB027F3FF455AE32
:1049640072E600BF00380240000047422DE9F341DF
:104974001D46174688460646FDF704FB3D442C1A9F
:10498400FDF700FB224B1B68C3F3CB33054663439F
:1049940032680193936838EA030301D000202DE0C4
:1049A4007B1CF7D0FDF7EEFA401BA04229D33368F5
:1049B4005A6822F0E0025A607268B2F5827F0AD126
:1049C400B268B2F5004F02D0B2F5806F03D11A6815
:1049D40022F040021A60B26AB2F5005F07D11A6889
:1049E40022F400521A601A6842F400521A60012339
:1049F40086F85130002386F85030032002B0BDE819
:104A0400F081019B002B019B08BF0024013BBFE701
:104A14000C00002038B513464268B2F5827F044684
:104A24001FD18268B2F5004F02D0B2F5806F07D172
:104A340025682868B2F5806F20F04000286007D010
:104A44000A4680212046FFF791FF20B9002038BD97
:104A54000A460121F6E7636D43F0200363650320F2
:104A6400F5E70A460121EEE737B51346124A156801
:104A7400124AB5FBF2F54FF47A7255434268019538
:104A8400B2F5827F04460BD10A468021FFF76EFF00
:104A940078B1636D43F020036365032003B030BD38
:104AA400019B33B1019B013B019323689B681B0667
:104AB400F6D40020F2E700BF0C00002000366E019F
:104AC40010B50446002855D0436A002B4ED14268E5
:104AD400B2F5827F00D0C3610023A36294F8513001
:104AE40003F0FF0223B984F850202046FCF728FB8A
:104AF4002168A068A269022384F851300B6823F06E
:104B040040030B60636800F4044003F482730343BE
:104B1400E06800F400600343206900F002000343EE
:104B2400606900F00100034302F400700343E0698C
:104B340000F038000343206A00F080000343A06AB9
:104B440000F4005003430B60636A120C03F010037B
:104B540002F004021A434A60CB6923F40063CB6178
:104B640000200123606584F8513010BD0023C0E9A2
:104B74000433B1E70120F8E72DE9F3411E4690F82C
:104B84005030012B04460D46174600F0A180012346
:104B940080F85030FDF7F6F994F85130012B804637
:104BA400D8B240F09380002D5ED0002F5CD0A26874
:104BB4002563032384F85130B2F5004F4FF000030E
:104BC4006365C4E91033E786A363A387E387A786F5
:104BD400236807D11A6822F040021A601A6842F466
:104BE40080421A601A68E16852065EBF1A6842F091
:104BF40040021A60B1F5006F626841D10AB1012F19
:104C040007D135F8022BDA602563E38E013B9BB2B2
:104C1400E386E38E9BB2A3B9424631462046FFF7B2
:104C240023FF00284FD1A36833B901932368DA68BE
:104C340001929B680193019B606D003818BF0120AD
:104C440012E022689368980705D5236B33F8021B9A
:104C5400D1602363D9E7FDF795F9A0EB0800B042D2
:104C64000BD3711CD5D00320012384F851300023C9
:104C740084F8503002B0BDE8F081002EC9D1F2E7CB
:104C84000AB1012F08D12A781A73236B01332363E5
:104C9400E38E013B9BB2E386E38E9BB2002BBBD039
:104CA40023689A68920702D5226B1278ECE7FDF725
:104CB40069F9A0EB0800B04202D3731CECD0D2E730
:104CC400002EE9D1CFE720236365ACE70220CBE7D0
:104CD4000220CFE72DE9F7431E4690F850300A9F93
:104CE400012B04460D46914600F0E680012380F82E
:104CF4005030FDF747F994F851306268012B804633
:104D0400D9B20AD0B2F5827F40F0D480A368002BD8
:104D140040F0D080042940F0CD80002D40D0B9F17E
:104D2400000F3DD0002E3BD094F85130C4F8389099
:104D3400042B1CBF052384F8513000236365C4E9A8
:104D440010332368E687E6861968A687490658BFA4
:104D54001968256358BF41F04001A68658BF196001
:104D6400E168B1F5006F52D10AB1012E07D135F8CF
:104D7400022BDA60E38E2563013B9BB2E3860125B7
:104D8400E38E9BB273B9E38F9BB25BB9424639465B
:104D94002046FFF769FE002800F081802023636528
:104DA40001202BE021688B689E070DD5E38E9BB212
:104DB40053B14DB1236B33F8022BCA602363E38EE6
:104DC400013B9BB2E38600258A6812F001020CD0F5
:104DD400E38F9BB24BB1A36BC96823F8021BA36397
:104DE400E38F013B9BB2E3871546FDF7CBF8A0EBBD
:104DF4000800B842C4D3781CC2D00320012384F82D
:104E04005130002384F8503003B0BDE8F0830AB178
:104E1400012E08D12A781A73236B01332363E38E9E
:104E2400013B9BB2E38601252DE022689368990734
:104E34000ED5E38E9BB25BB155B1236B1B78137314
:104E4400236B01332363E38E013B9BB2E38600258E
:104E54002268916811F001010DD0E38F9BB253B128
:104E6400A36BD2681A70A36B0133A363E38F013B76
:104E74009BB2E3870D46FDF785F8A0EB0800B84226
:104E84000AD37B1CB9D1E38E9BB2002BCDD1E38F27
:104E94009BB2002BC9D179E7002FF4D1ADE7A36809
:104EA400002BABD123680190DA6801929B680193CF
:104EB400019BA3E70220A1E70220A5E72DE9F74320
:104EC4001D464368B3F5827F0446894617460CD1D4
:104ED400836853B9042380F85130134600950A4679
:104EE400FFF7F8FE03B0BDE8F08394F85030012BCF
:104EF40000F08680012384F85030FDF743F894F8DD
:104F04005130012B8046D8B278D1B9F1000F5CD072
:104F1400002F5AD0A268C4F8389000260423B2F5B2
:104F2400004F84F85130C4E9106666652368E7874A
:104F3400A7872663A686E68607D11A6822F0400270
:104F44001A601A6822F480421A601A6856065EBF14
:104F54001A6842F040021A60E368F3B1E38F9BB22F
:104F6400FBB123689A68D20739D5DA68A36B23F8B2
:104F7400022BA363E38F013B9BB2E387EEE7236835
:104F84009A68D00718D5A26B1B7B1370A36B0133EF
:104F9400A363E38F013B9BB2E387E38F9BB2002BB8
:104FA400EDD1424629462046FFF734FD18BB606D1B
:104FB400003818BF012008E0FCF7E4FFA0EB08006C
:104FC400A84209D3691CE8D00320012384F8513096
:104FD400002384F8503085E7002DDED1F4E7FCF798
:104FE400D1FFA0EB0800A84202D36B1CB6D0EBE7BC
:104FF400002DB3D1E8E720236365D8E70220E4E776
:1050040002206FE7036A23F001030362036A70B5A9
:10501400446882690D6822F073022A438D6823F084
:1050240002032B430E4DA84202D00E4EB04210D1C3
:10503400CE6823F008033343A84223F0040302D0CC
:10504400084DA84205D1D1E9055624F440743543EE
:105054002C43446082614A684263036270BD00BFAE
:105064000000014000040140036A23F480730362DA
:10507400036A70B54468C2690D6822F073022A435A
:105084008D6823F4007343EA0523114DA84203D02D
:1050940005F58065A84214D1CD6823F4006343EA82
:1050A40005230B4DA84223F4806303D005F58065E6
:1050B400A84206D1D1E9055624F44054354344EAC4
:1050C40005144460C2614A68C263036270BD00BFD4
:1050D40000000140036A23F480530362036A30B57D
:1050E4004468C2690D6822F4E64242EA05228D68EA
:1050F40023F4005343EA0533084DA84203D005F5D1
:105104008065A84204D14D6924F4804444EA85149E
:105114004460C2614A680264036230BD0000014019
:1051240090F83D30012B30D1022380F83D300368E4
:10513400DA6842F00102DA60154A93421AD0B3F1F8
:10514400804F17D0A2F57C42934213D002F58062BF
:1051540093420FD002F5806293420BD002F578425D
:10516400934207D002F57052934203D0A2F59432D1
:10517400934204D19A6802F00702062A03D01A68FF
:1051840042F001021A60002070470120704700BFFE
:1051940000000140704770477047704770470368CC
:1051A4001A69910710B504460ED5DA6892070BD533
:1051B4006FF002021A61012202779B699B0777D084
:1051C400FFF7EAFF0023237723681A69500710D5F5
:1051D400DA6851070DD56FF004021A6102222277B2
:1051E4009B6913F4407F204668D0FFF7D5FF002366
:1051F400237723681A6912070FD5DA6810070CD5CC
:105204006FF008021A6104222277DB6999072046AD
:105214005AD0FFF7C1FF0023237723681A69D20607
:1052240010D5DA68D0060DD56FF010021A61082285
:105234002277DB6913F4407F20464BD0FFF7ACFFA5
:105244000023237723681A69D10708D5DA68D207BF
:1052540005D56FF001021A612046FBF7CDFE2368E5
:105264001A69100608D5DA68110605D56FF08002B0
:105274001A61204600F009FB23681A69520608D512
:10528400DA68500605D56FF040021A612046FFF730
:1052940085FF23681A69910622D5DA6892061FD51C
:1052A4006FF0200220461A61BDE8104000F0ECBA0D
:1052B400FFF771FF2046FFF770FF83E7FFF76BFFEF
:1052C4002046FFF76AFF92E7FFF765FF2046FFF7E6
:1052D40064FFA0E7FFF75FFF2046FFF75EFFAFE73D
:1052E40010BD0000304A0368904212D0B0F1804FE4
:1052F4000FD0A2F57C4290420BD002F5806290421E
:1053040007D002F58062904203D002F578429042C1
:1053140019D14A6823F070031343234A904229D0D9
:10532400B0F1804F26D0A2F57C42904222D002F503
:10533400806290421ED002F5806290421AD002F53B
:105344007842904216D0194A904213D002F58062F6
:1053540090420FD002F5806290420BD0A2F59832B1
:10536400904207D002F58062904203D002F5806239
:10537400904203D1CA6823F4407313434A6923F06B
:105384008003134303608B68C3620B688362064B1C
:10539400984203D003F58063984201D10B690363FB
:1053A40001234361704700BF0000014000400140F9
:1053B40010B5044630B390F83D3003F0FF021BB93A
:1053C40080F83C20FCF7C8F80223206884F83D30BC
:1053D400211DFFF787FF012384F84630002084F85D
:1053E4003E3084F83F3084F8403084F8413084F80B
:1053F400423084F8433084F8443084F8453084F8EB
:105404003D3010BD0120FCE710B5044630B390F8E0
:105414003D3003F0FF021BB980F83C20FFF7BAFED1
:105424000223206884F83D30211DFFF75BFF012330
:1054340084F84630002084F83E3084F83F3084F805
:10544400403084F8413084F8423084F8433084F8A2
:10545400443084F8453084F83D3010BD0120FCE729
:10546400036A23F010030362036A70B54468826917
:105474000D6822F4E64242EA05228D6823F02003F7
:1054840043EA0513104DA84203D005F58065A842F0
:1054940014D1CD6823F0800343EA05130A4DA842D2
:1054A40023F0400303D005F58065A84206D1D1E975
:1054B400055624F44064354344EA8504446082611B
:1054C4004A688263036270BD0000014070B590F8C1
:1054D4003C30012B054653D00120082A85F83C00B6
:1054E4003DD006D8C2B1042A28D0002385F83C3028
:1054F40070BD0C2AF9D12868FFF7ECFD2B68096907
:10550400DA6942F40062DA61DA6922F48062DA610B
:10551400DA6942EA012231E02868FFF773FD2B685B
:1055240009699A6942F008029A619A6922F00402B0
:105534009A619A690A439A610020D6E72868FFF7BE
:105544008FFF2B6809699A6942F400629A619A692B
:1055540022F480629A619A6942EA0122EBE72868A0
:10556400FFF782FD2B680969DA6942F00802DA6103
:10557400DA6922F00402DA61DA690A43DA61DBE704
:105584000220B5E710B58468114324F47F4441EA4E
:1055940003232343836010BD70B590F83C30012B86
:1055A40004464FF0020300F09180012280F83D3060
:1055B40080F83C200068836823F47F4323F077035A
:1055C40083600B68602B52D033D8402B67D016D839
:1055D400202B0DD00AD833F0100109D0012384F810
:1055E4003D30002384F83C30104670BD302BF5D19B
:1055F400826822F07002134343F0070317E0502B34
:10560400ECD14A68CE68016A056A25F00105056295
:10561400836921F00A0123F0F00343EA06130A43E5
:1056240083610262836823F0700343F0570383604D
:1056340011E0B3F5805F0ED0B3F5005F0DD0702B91
:10564400CCD1CB68D1E90121FFF79CFF2268936894
:1056540043F0770393600022C0E7CB68D1E90121CE
:10566400FFF790FF2268936843F48043F2E74D68A4
:10567400CE68016A21F0100101628269036A22F492
:10568400704223F0A00343EA051342EA0632826122
:105694000362836823F0700343F06703C7E74A6833
:1056A400CE68016A056A25F001050562836921F067
:1056B4000A0123F0F00343EA06130A4383610262FA
:1056C400836823F0700343F04703B0E71A468BE77F
:1056D400036A01F01F0110B501248C4023EA04037E
:1056E4000362036A8A401A43026210BD10B504467D
:1056F40029B990F83E30012B18D001202DE004295F
:105704000DD190F83F30013B18BF0123002BF4D199
:1057140004294FF0020321D184F83F3009E008291D
:105724000CBF90F8403090F84130ECE7022380F849
:105734003E3020680122FFF7CBFF23681C498B42CF
:1057440013D01C4A934210D0B3F1804F14D19A68FD
:1057540002F00702062A26D1002010BD08290CBF3A
:1057640084F8403084F84130E3E75A6C8B4242F4C9
:1057740000425A64EBD0E7E70F4A9342E7D002F5C0
:1057840080629342E3D002F580629342DFD002F557
:1057940078429342DBD002F570529342D7D0A2F5FF
:1057A40094329342D3D01A6842F001021A60D3E7CC
:1057B400000001400004014000040040FFF796BFD0
:1057C40030B590F83C30012B4FF0020332D080F812
:1057D4003D3003680D685C689A6824F070042C43BB
:1057E4005C60154CA3421AD0B3F1804F17D0A4F5D6
:1057F4007C44A34213D004F58064A3420FD004F583
:105804008064A3420BD004F57844A34207D004F586
:105814007054A34203D0A4F59434A34204D149683C
:1058240022F080020A439A60012380F83D3000236D
:1058340080F83C30184630BD0000014090F83C3000
:10584400012B1FD0CB688A6823F4407313434A6842
:1058540023F4806313430A6823F4006313430A693F
:1058640023F4805313434A6923F400531343CA694E
:1058740023F48043134302685364002380F83C30CC
:10588400184670470220704770477047026802F15B
:105894000C0353E8003F23F490730C3242E80031C8
:1058A40002680029F2D102F1140353E8003F23F007
:1058B400010302F1140C4CE800310029F3D1036B0D
:1058C400012B0BD102F10C0353E8003F23F010032A
:1058D40002F10C0C4CE800310029F3D1202380F8AC
:1058E4003E300023036370470268C168136923F4E0
:1058F40040530B4370B51361054683680069D16852
:10590400034368690343E86921F4164121F00C015B
:1059140003430B43D3605369A96923F440730B43D6
:1059240053611F4B9A4203D003F580639A4223D1FB
:10593400FEF7D6FBEB691921B3F5004FD5E9004614
:10594400A0FB01011BD1B2194FF000035B41FAF730
:105954005FFC6421B0FBF1F501FB1503DB0032337E
:10596400B3FBF1F303F007025B0002EB051203F44F
:10597400F8731344A36070BDFEF7A2FBDAE7B2002C
:10598400B30FFAF745FC6422B0FBF2F102FB1103FA
:105994001B013233B3FBF2F303EB0113EAE700BF5D
:1059A4000010014010B5044640B390F83D3003F0B8
:1059B400FF021BB980F83C20FCF762F9226824231B
:1059C40084F83D30D36823F40053D3602046FFF7B6
:1059D4008BFF23681A6922F490421A615A6922F0F3
:1059E4002A025A61DA6842F40052DA600020202365
:1059F400206484F83D3084F83E3010BD0120FCE77B
:105A040038B50446134694F83D20202A32D179B3A0
:105A140073B394F83C20012A2CD0012284F83C2052
:105A2400606BE38400252122256484F83D20124A1A
:105A3400A3842162C263114A0264114AC0E9132596
:105A440022680432FCF7B0FE23686FF040021A604B
:105A5400226884F83C5002F1140353E8003F43F0F9
:105A6400800302F1140141E800300028F3D138BD6D
:105A74000120FCE70220FAE7895A0008D75A0008F7
:105A8400E55A000808B50346806B1B681B6813F4CD
:105A940080731AD1C384026802F1140353E8003FEF
:105AA40023F08003143242E8003102680029F2D165
:105AB40002F10C0353E8003F43F0400302F10C00F1
:105AC40040E800310029F3D108BDFCF751F9FBE7A8
:105AD400704708B5806BFFF7FBFF08BD7047704740
:105AE40008B5806B03685A6990F83D10212912D1DA
:105AF400120610D50022C28403F10C0252E8002FD2
:105B040022F0C00203F10C0C4CE800210029F3D16F
:105B1400202280F83D205B6990F83E20222A05D19E
:105B24005B0603D50023C385FFF7B0FE036C43F087
:105B340010030364FFF7D3FF08BD08B5806B00238F
:105B4400C385C384FFF7CBFF08BD7047806B08B5DE
:105B5400036B012B04D1818D4908FFF7F6FF08BDC3
:105B6400FFF7BCFFFBE708B50346806B1B681B68A7
:105B740013F4807337D1C385026802F10C0353E830
:105B8400003F23F480730C3242E80031036800299B
:105B9400F2D103F1140252E8002F22F0010203F1C2
:105BA400140C4CE800210029F3D103F1140252E84B
:105BB400002F22F0400203F1140C4CE800210029CC
:105BC400F3D1202280F83E20026B012A0BD103F18D
:105BD4000C0252E8002F22F0100203F10C0C4CE8E6
:105BE40000210029F3D1036B012B03D1818DFFF731
:105BF400ACFF08BDFCF7D0F8FBE707B58168836A02
:105C04000268B1F5805F3ED1016900293ED1526836
:105C1400C2F3080223F8022B8362C38D013B9BB2BB
:105C2400C385002B2CD10268D16821F02001D160FA
:105C3400D16821F48071D160516921F00101516171
:105C4400202280F83E20026B012A026828D10363D7
:105C540002F10C0353E8003F23F0100302F10C0C93
:105C64004CE800310029F3D11368DB0605D5019116
:105C74001368019353680193019B818DFFF765FFBE
:105C840003B05DF804FB39B9016929B95268D2B28D
:105C94001A70836A0133BFE7526802F07F02F7E7A4
:105CA400FCF77AF8ECE70000036837B51A68D9689E
:105CB4005D6912F00F0F04460CD1950670D58D0660
:105CC4006ED590F83E30222B64D103B0BDE830404D
:105CD400FFF793BF05F0010001F4907505435FD011
:105CE400D50705D5CB0542BF236C43F001032364DC
:105CF400550704D518B1236C43F0020323649307BA
:105D040004D518B1236C43F004032364150707D5A5
:105D140001F0200303431EBF236C43F008032364F4
:105D2400236C002B36D0900608D58A0606D594F845
:105D34003E30222B02D12046FFF75FFF23685B69C8
:105D4400256C03F0400305F008051D43204623D0CD
:105D5400FFF79CFD226853695B0618D502F1140312
:105D640053E8003F23F0400302F1140040E80031FF
:105D74000029F3D1A06B50B1724B0365FCF792FD7F
:105D840040B1A06B036D03B0BDE830401847204616
:105D9400FFF7A5FE03B030BDFFF7A1FE2564F9E7C8
:105DA400206B012840F09180D50640F18E80C80612
:105DB40040F18B80002201921A6801925A68019284
:105DC400019A5A6955064CD5A16B0A68526892B279
:105DD400002ADFD0A08D9042DCD9E285CA69B2F5F1
:105DE400807F36D003F10C0252E8002F22F4807237
:105DF40003F10C0040E800210029F3D103F114025F
:105E040052E8002F22F0010203F1140040E80021BF
:105E14000029F3D103F1140252E8002F22F04002CA
:105E240003F1140040E800210029F3D1202284F872
:105E34003E20216303F10C0252E8002F22F01002ED
:105E440003F10C0040E800210029F3D1A06BFCF71A
:105E5400E5FCE38DA18DC91A89B22046FFF775FED2
:105E640098E7E18D8AB2E18D89B2002992D0A18DA3
:105E7400891A89B200298DD003F10C0252E8002F4F
:105E840022F4907203F10C0545E800200028F3D1B8
:105E940003F1140252E8002F22F0010203F1140569
:105EA40045E800200028F3D1202284F83E20206316
:105EB40003F10C0252E8002F22F0100203F10C054A
:105EC40045E800200028F3D1C7E7100628D50D06C1
:105ED40026D594F83D20212A7FF45CAFA168226A7C
:105EE400B1F5805F17D12169A9B932F8021BC1F35A
:105EF400080159602262E28C013A92B2E284002ADB
:105F04007FF448AFDA6822F08002DA60DA6842F09F
:105F14004002DA603EE7511C216212785A60EAE7D7
:105F240050067FF537AF4A067FF534AFDA6822F0C2
:105F34004002DA60202384F83D302046FBF718FF46
:105F440028E700BF3F5B000873B522230025044601
:105F54000564816280F83E308285806B1E4BC3638A
:105F64001E4B266803641E4BC0E9133513460A46CC
:105F7400311DFCF719FC236801951A6801925A68CF
:105F84000192019A226984F83C505AB103F10C023F
:105F940052E8002F42F4807203F10C0040E8002123
:105FA4000029F3D103F1140252E8002F42F0010258
:105FB40003F1140040E800210029F3D103F1140295
:105FC40052E8002F42F0400203F1140141E800209E
:105FD4000028F3D102B070BD6B5B0008515B000870
:105FE400E55A000870B490F83E60202E10D161B1DB
:105FF4005AB190F83C40012C0AD0012480F83C406E
:106004000024046370BCFFF79FBF012070BC70477D
:106014000220FBE782B00023104A0193019B013365
:106024000193019B934216D80369002BF6DA0023EF
:1060340001930369094A43F001030361019B01339E
:106044000193019B934206D8036913F00103F5D130
:10605400184602B070470320FBE700BF400D030061
:1060640084B038B505AD85E80E000A9B012B0446C3
:1060740025D1836B23F480338363C36823F48403BF
:1060840023F04003C360C36823F44013C360119B2F
:10609400012B02BFC36843F48013C360FFF7BAFF48
:1060A400089B012B07D1A36843F00603A360A368F0
:1060B40043F02003A360BDE8384004B07047C368D0
:1060C40043F04003C360FFF7A5FF0E9B23B9A36B06
:1060D40043F48033A363E3E7A36B23F48033F9E74A
:1060E400022A4AD1274B284A0B44934239D9274BD9
:1060F400274A0B44934236D9264AA1F57403A3F5E3
:106104001053934231D9244AA1F18373A3F5E74391
:1061140093422CD3214B224A0B44934229D9214B3D
:10612400214A0B44934226D3204B214A0B449342E9
:1061340023D3204AA1F1B773A3F5585393421ED336
:106144001D4B1E4A0B44934234BF07230623C268E7
:1061540022F47052C260C26842EA8323C360002002
:1061640070470F23F3E70E23F1E70D23EFE70C232A
:10617400EDE70B23EBE70A23E9E70923E7E7082325
:10618400E5E700BF405327FFFF340C00401E1BFF10
:106194003F420F007F4F120020D6130060B6E5FE89
:1061A4005FE3160000D3CEFE40771B00C05BB3FE56
:1061B400C091210020753800E05459FEE09C410054
:1061C400836843F00103836000207047836823F0F1
:1061D400010383600020704738B5C368012923F0A8
:1061E400C0430546C36010D1C36843F00053C36085
:1061F40000240120FBF7CCFE6B69D90704F10104EC
:1062040015D4322CF5D1012038BD0029FBD1C36847
:1062140043F08043C3600C460120FBF7B9FE6B6971
:10622400DA0704F1010402D5322CF5D1EBE7A4F12D
:10623400320358425841E7E782B00023104A0193E1
:10624400019B01330193019B934216D80369002BF0
:10625400F6DA8901002341F02001094A0193016122
:10626400019B01330193019B934206D8036913F008
:106274002003F5D1184602B070470320FBE700BFA6
:10628400400D030082B000230F4A0193019B0133A8
:106294000193019B934214D80369002BF6DA00237F
:1062A4000193094A10230361019B01330193019B6C
:1062B400934206D8036913F01003F5D1184602B0CF
:1062C40070470320FBE700BF400D0300D0F80038FF
:1062D4001943C0F8001800207047000084B02DE96D
:1062E400F843044609A880E80E00139D00230E46D7
:1062F400194603F1400204EB820201330F2B516073
:10630400F7D104F50067002D6CD17B6843F00203DC
:106314007B60A36B23F40013A363236843F040035F
:106324002360236843F0800323600023C4F8003E05
:10633400D4F80038C4F800380E9B012B59D10B99BE
:10634400002954D12046FFF7C1FF10212046FFF752
:1063540073FF01462046FFF795FF0843C0B20023B0
:1063640000383B6118BF01207B6104F51062FB61BA
:1063740019464FF0904C4FF0006E4FF67F38B34201
:1063840039D1002204F5306311464FF0904C4FF0A0
:10639400006E4FF67F38B24240D13B6923F48073DC
:1063A4003B610023A3616FF0804363610C9B1BB9C5
:1063B400A36943F01003A361A269224B1343A361B1
:1063C4000F9B1BB1A36943F00803A361012D01BF17
:1063D400A36943F0804343F00403A361BDE8F84399
:1063E40004B07047A36B43F40013A3639DE71946FD
:1063F400A8E70321A6E7D2F80090B9F1000F0BDA61
:106404003BB9C2F800E011610133C2F808802032C0
:10641400B5E7C2F800C0F6E71160F4E7D3F80090DE
:10642400B9F1000F0BDA3AB9C3F800E0196101328F
:10643400C3F808802033AEE7C3F800C0F6E719605C
:10644400F4E700BF00383C80D0F8083813F00600A9
:1064540004D013F0020F14BF02200F20704730B590
:106464000D78012405F00F039C404B7800F5006281
:10647400012B00EB4510D36918D11C43D461D0F82B
:1064840000391A0410D4CA68D0F80049C2F30A03C8
:106494000A79234343EA824343EA855343F0805312
:1064A40043F40043C0F80039002030BD43EA0444FB
:1064B400D461D0F8003B1B04F6D4CB68D0F8002B91
:1064C400C3F30A0313430A7943EA824343F0805334
:1064D40043F40043C0F8003BE6E7000010B50A7837
:1064E4004978012900EB421300F5006002F00F0225
:1064F40022D1D3F8001900290BDAD3F8001941F09E
:106504000061C3F80019D3F8001941F08041C3F8C1
:106514000019C46B012101FA02F224EA0204C463E3
:10652400C16921EA0202C261D3F80019144A0A407F
:10653400C3F80029002010BDD3F8001B00290BDA92
:10654400D3F8001B41F00061C3F8001BD3F8001B13
:1065540041F08041C3F8001BC46B4FF4803101FA51
:1065640002F224EA0204C463C16921EA0202C2619C
:10657400D3F8001B034A0A40C3F8002BDAE700BF34
:10658400007833EC0078F3EF4B78DFF8F0C0F0B527
:106594000E788D69384F012B00EB461446D104F573
:1065A4001063BDB91D692F401F611D6945F40025A5
:1065B4001D611D6905EA0C05012A1D6123D14A6983
:1065C40002B15A61D4F8003943F00443C4F80039E5
:1065D4000020F0BDD3F810E00EEA0C0CC3F810C094
:1065E400D3F810C00CEA07071F61CF68AF421D69DA
:1065F40038BF8F6145F400251D618D691F69C5F39E
:1066040012053D43D8E7D4F8003943F00443C4F8F5
:1066140000398B69002BDBD0D0F8342806F00F0644
:106624000123B3401343C0F83438D1E7D4F8100B36
:1066340000EA0C00C4F8100BD4F8100B384004F531
:1066440030631861C86805B188611D69C86145F483
:1066540000251D611D69C0F312002843012A186139
:1066640002D10A6902B15A61D4F8003B43F00443F1
:10667400C4F8003BACE700BFFFFF07E00000F8FFF1
:1066840082B000234A7801930B78012A4FEA43131E
:106694001ED100F51060C118C258002A02DB002088
:1066A40002B07047C25842F00062C250C25842F071
:1066B4008042C25042F21072019B01330193019B4C
:1066C400934201D90120EBE70B68002BF4DBE6E7EA
:1066D40000F53060C118C258002AE0DAC25842F00E
:1066E4000062C250C25842F08042C25042F210725C
:1066F400019B01330193019B9342E3D80B68002B68
:10670400F6DBCCE710B59DF8084044B903330132F9
:106714009B0800EB023001EB83038B4201D1002084
:1067240010BD51F8042B0260F7E700002DE9F34196
:106734004D780F788B690E79DFF8BCC1DFF8BCE1C6
:10674400012D00EB471440F08E8004F51065D5F858
:1067540010806BBB08EA0C0CC5F810C0D5F810C04B
:106764004CF4002CC5F810C0D5F810C00CEA0E0E7D
:10677400C5F810E0012A4ED14B6903B16B61012EBB
:106784000CD1D0F8083813F4807FD4F800390CBF4A
:1067940043F0005343F08053C4F80039D4F800396F
:1067A40043F00443C4F80039002002B0BDE8F0818E
:1067B40008EA0E0EC5F810E0D5F810E00EEA0C0C4D
:1067C400D1F80CE0C5F810C00EEB030C0CF1FF3C43
:1067D400BCFBFEFEDFF828C1D5F810800CEACE4CD5
:1067E4004CEA080CC5F810C0D5F810E0C3F3120C3D
:1067F4004CEA0E0C012EC5F810C0BBD1D5F810C060
:106804002CF0C04CC5F810C0D5F810C04CF0005C9A
:10681400C5F810C0AEE7D4F80059012E45F0044580
:10682400C4F800590BD0002BBED0D0F8343807F090
:106834000F02012797401F43C0F83478B4E7D0F81B
:10684400085815F4807FD4F800590CBF45F0005562
:1068540045F08055C4F80059009209699BB23A4644
:10686400FFF750FFA0E7D4F8105B05EA0E05C4F863
:10687400105BD4F8105B05EA0C0504F530673D6144
:10688400CD681BBB3B69C5F312051D433D613B69E4
:1068940043F400233B61012A02D10B6903B17B61FC
:1068A400012E0CD1D0F8083813F4807FD4F8003BC3
:1068B4000CBF43F0005343F08053C4F8003BD4F8BA
:1068C400003B43F00443C4F8003B6DE72B44DFF87E
:1068D40030C0D7F810E0013BB3FBF5F39BB25D4346
:1068E4000CEAC34343EA0E03CD613B613B69C5F344
:1068F40012051D433D61CEE7FFFF07E00000F8FFEE
:106904000000F81F034670B59008002402F003024B
:1069140003F58055844210D301EB800062B103F586
:1069240080531C680023D90024FA01F1C1540133B7
:1069340099B28A42F7D1104470BD2E6841F82460A0
:106944000134E7E74A780B78012A00EB431012D1AF
:10695400D0F80029002A06DB2BB1D0F8003923F047
:106964008043C0F80039D0F8003943F40013C0F86C
:10697400003900207047D0F8002B002A06DB2BB129
:10698400D0F8003B23F08043C0F8003BD0F8003B34
:1069940043F40013C0F8003BEBE70B784A7800EBB4
:1069A40043100B79012AA3F10203DBB20FD1D0F813
:1069B4000029012B22F40012C0F8002905D8D0F8D0
:1069C400003943F08053C0F8003900207047D0F8F4
:1069D400002B22F40012012BC0F8002B9EBFD0F82C
:1069E400003B43F08053C0F8003BEEE7D0F800389A
:1069F40023F4FE63C0F80038D0F80038090101F42C
:106A0400FE611943C0F8001800207047D0F8003E1A
:106A140023F00303C0F8003ED0F8043823F0020347
:106A2400C0F8043800207047D0F8003E23F0030378
:106A3400C0F8003ED0F8043843F00203C0F804382C
:106A4400002070474269806910407047D0F81838B8
:106A540000F50060C0691840000C7047D0F8183881
:106A640000F50060C069184080B2704700EB411126
:106A740000F50060D1F8082B40691040704710B54C
:106A8400D0F81048D0F8343800EB411001F00F0171
:106A9400CB4000F51060DB018068DBB22343184073
:106AA40010BD406900F001007047D0F8003923F4AC
:106AB400FF6323F00703C0F80039D0F8043843F427
:106AC4008073C0F8043800207047000030B5056CAE
:106AD400104CA54200F5306303D9D0F8004B002CCC
:106AE40016DB00241C611C6944F400241C611C692D
:106AF40044F018041C611C69012944F0C0441C6161
:106B040001BF5A61D0F8003B43F08023C0F8003B3A
:106B1400002030BD0A30544FD0F8D43200EB83004B
:106B240010B5D0F8C04284B1D0F8C4325BB194F847
:106B34000002FF2807D09B6894F801222146984759
:106B4400FF2384F80032002000E0032010BD000081
:106B54000A230380004870479400002070B5822106
:106B640006460F4800F079FB012105460C4800F069
:106B740074FB812104460A4800F06FFB0DB110221A
:106B8400AA711CB1402222710022627118B1402204
:106B940002710022427143230148338070BD00BF5B
:106BA40050000020FFF7DABF70B5822106460F4877
:106BB40000F053FB012105460C4800F04EFB8121F7
:106BC40004460A4800F049FB0DB11022AA711CB119
:106BD400002222710222627118B100220271022283
:106BE400427143230148338070BD00BF5000002030
:106BF40038B5D0F8D432B033044650F823508DB1B0
:106C040000F0B9FFC5F80C02D4F8D40204EB8004F8
:106C140005F50371D4F8C432D5F80402DB6898474B
:106C2400002038BD0320FCE7F8B5D0F8D46200EBAF
:106C340086060A46D6F8C05245B301F00F0C142755
:106C440007FB0C07BC6994B1D0F8C8324FF0240E8E
:106C54000EFB0C339B6CB4FBF3FC03FB1C4434B9F8
:106C6400BC612346224601F004F820460DE0D6F824
:106C7400C4321C690027C5F81472002CF5D0D5F86D
:106C8400080205F50471A0473846F8BD0320FCE767
:106C9400D0F8D4322DE9F34100EB83034FF0000820
:106CA400D3F8C0728DF8058005460E46ADF806800F
:106CB400002F6ED00A7812F060042ED0202C64D1FC
:106CC400CC8891F801C00CB3120613D5D3F8C432A2
:106CD400224639469B6860469847F288072A28BFAF
:106CE40007223946284600F032FD4446204602B0C9
:106CF400BDE8F081402C28BF402487F800C287F803
:106D040001422246394600F037FDEEE7D3F8C4329B
:106D140022469B6860469847E8E74F780B2F34D8A3
:106D240001A353F827F000BF5D6D0008F16C000863
:106D34008F6D00088F6D00088F6D00088F6D00083F
:106D44008F6D00088F6D00088F6D00088F6D00082F
:106D5400736D0008876D000890F89C32032B14D1E2
:106D640002220DF1060100F0F2FC3C46BEE790F869
:106D74009C32032B09D101220DF1050100F0E7FC3F
:106D8400B4E790F89C32032BB0D03146284600F08B
:106D9400B7FC0324AAE700BF38B5044600258121C7
:106DA40000F043FF01212587204600F03EFFA4F8B0
:106DB40078518221204600F038FFD4F8D432E564BB
:106DC40004EB8303D3F8C0228AB1D3F8C4325B68DE
:106DD4009847D4F8D432B03354F8230000F006FFB7
:106DE400D4F8D432B03344F82350C4F8BC52002051
:106DF40038BD70B504464FF4077000F0F3FE054645
:106E040030B9D4F8D432B03344F82300022547E033
:106E14004FF40772002100F063FFD4F8D432B0338A
:106E240044F82350237CC4F8BC52002B3AD14FF4CD
:106E34000073022281212046012600F0EAFE268703
:106E44004FF4007331460222204600F0E2FE102384
:106E54000322A4F87861A4F84E3082210823204646
:106E640000F0D7FED4F8D43204EB83030026D3F821
:106E7400C4320121A4F84C101B68C5F80462984779
:106E8400D5F80422C5F81462C5F81862002ABDD0EA
:106E9400257C012185B94FF40073204600F0F2FEF1
:106EA400284670BD4023022281212046012600F09D
:106EB400B0FE26874023C5E74023204600F0E2FECB
:106EC4003546EDE739B1D0F8D43200EB8300C0F891
:106ED400C4120020704703207047D0F8D432B03376
:106EE40050F823302BB1C3F80812C3F81022002045
:106EF400704703207047D0F8D432B03350F82330B1
:106F04001BB1C3F804120020704703207047D0F867
:106F1400D422B03210B550F8222082B1047CD2F8C9
:106F2400042234B94FF40073012100F0ABFE204673
:106F340010BD4023012100F0A5FE0024F7E703243F
:106F4400F5E778B10023C0F8B832C0F8C432C0F80D
:106F5400D03209B1C0F8B412012380F89C32027017
:106F640000F0C8BD0320704713B500230446ADF8F4
:106F7400063081B1CB6AC0F8B81223B10DF1060016
:106F84009847C4F8D002D4F8D8320133C4F8D832C0
:106F9400002002B010BD0320FBE700F031BED0F8A2
:106FA400B8320BB11B6818471846704708B5D0F8BB
:106FB400B8325B689847002818BF032008BD38B56D
:106FC400044600F2AA25284600F08FFB012394F81A
:106FD400AA12C4F89432B4F8B032C4F8983201F06A
:106FE4001F03012B08D0022B0CD08BB92946204655
:106FF400BDE8384000F04EB929462046BDE8384087
:1070040000F0A6BA29462046BDE8384000F0CFBAC1
:10701400204601F08001BDE8384000F00FBE70B595
:107024000446164609BBD0F89432032B0CD1D0E9A0
:10703400573293420AD99B1A9A42C0F85C3128BF4E
:107044001A46314600F0A5FB002070BD90F89C3232
:10705400032B06D1D0F8B8321B6913B1C0F8D4128F
:107064009847204600F09DFBEEE790F89C32032BF6
:10707400EAD1D0F8B8329B69002BE5D00022BDE8F4
:107084007040C0F8D422184773B504461646002948
:1070940041D1D0F89422022A0FD1D0E90752954267
:1070A40014D9AA1A0191C261314600F05DFB019B1B
:1070B4001A461946204600F0E5FD94F8A03213B1B3
:1070C400002384F8A032002002B070BD0ED1826982
:1070D40095420BD8D0F89852AA4207D20A46019199
:1070E40000F042FB019BC4F89832E1E794F89C322B
:1070F400032B08D1D4F8B832DB6823B10022C4F8DA
:10710400D422204698478021204600F097FD20464F
:1071140000F052FBD1E790F89C32032BD3D1D0F886
:10712400B8325B69002BCED00022C0F8D42202B062
:10713400BDE870401847F8B5012380F89C32D0F8B8
:10714400B83200210446C0F894124160C0F8A41279
:1071540080F8A012B3B90026002240251146012769
:107164004023204600F055FDA4F86471C4F8605132
:107174002B4600228021204600F04BFDA784256287
:107184003046F8BD5B68002BE5D098470028E2D074
:107194000326E1E701740020704790F89C32DBB2CB
:1071A40080F89D32042380F89C320020704790F8C8
:1071B4009C32042B02BF90F89D32DBB280F89C32E3
:1071C4000020704708B590F89C22032A05D1D0F816
:1071D400B83213B1DB6903B19847002008BDD0F879
:1071E400D422AE3208B550F8222042B190F89C3235
:1071F400032B02D1136A23B19847002000E0032037
:1072040008BD1846FCE7D0F8D422AE3208B550F8D1
:10721400222042B190F89C32032B02D1536A23B14D
:107224009847002000E0032008BD1846FCE7002032
:107234007047012208B580F89C22D0F8B8220AB918
:10724400002008BD5268017990470028F8D0032037
:10725400F7E7002070470020704710B54288037894
:107264009A420AD90478204423444478052C9BB2DA
:10727400F6D184788C42F3D110BD0020FCE710B520
:107284008021044600F0DAFC20460021BDE81040CD
:1072940000F0D4BC2DE9F3410D7805F06005202DF4
:1072A40004460E4614D0402D12D0002D40F0128119
:1072B4004F78092F00F20E81DFE817F013013C012B
:1072C4000C012B010C018E0016000C01FB00AA001E
:1072D400D4F8D432AE33314654F823309B68204678
:1072E40002B0BDE8F04118470023ADF806304B88E2
:1072F4001A0A013A0E2A0DD8DFE802F0132C390CD1
:107304000C59630C0C0C0C0C0C0C0800D0F8B432A7
:10731400DB694BB92046FFF7B2FF284602B0BDE84F
:10732400F081D0F8B4321B68207C0DF10601984737
:10733400F288002A00F0FA80BDF80630002BE9D06C
:107344009A4228BF1A46ADF806200146204600F0AE
:10735400FEF9E2E7027CD0F8B83232B99B6A0DF14B
:107364000600984702234370E2E7DB6AF7E7DBB2E3
:10737400052BCFD8DFE803F003070B0F1317D0F862
:10738400B4325B68C5E7D0F8B4329B68C1E7D0F883
:10739400B432DB68BDE7D0F8B4321B69B9E7D0F882
:1073A400B4325B69B5E7D0F8B4329B69B1E7037CCA
:1073B400002BAFD1D0F8B8320DF106005B6B9847C3
:1073C400B6E7037C002BA5D1D0F8B8320DF1060046
:1073D4001B6B98470723C6E78B88002B9AD1CB8871
:1073E400002B97D14E887F2E94D890F89C32032B93
:1073F40090D0F1B280F89E1200F032FC204600F0EA
:10740400D0F91EB1022384F89C3286E70123FAE7FF
:107414008E784E4F012E3E7003D9FFF730FF0325BF
:107424007BE790F89C32022B5FFA83F809D0B8F11D
:10743400030F18D0FFF723FF39782046FFF7B6FD76
:10744400EDE7002E72D001214160FFF7A8FD05464B
:10745400204625B1FFF713FF84F89C825DE700F016
:10746400A0F90323CFE75EB9022380F89C3246607B
:107474003146FFF79BFD204600F093F935464CE773
:107484004168012952D0C9B2FFF790FD3978616093
:107494002046FFF784FD0646002847D02046FFF724
:1074A400EEFE21792046FFF781FD022384F89C3209
:1074B400E4E7CA88012A7FF42DAF90F89C120229D0
:1074C400CBB205D833B10146002341F8083F3DE76C
:1074D400032B04D02046FFF7D2FE00251DE7011D33
:1074E40034E790F89C32013B022BF3D8CB88022B73
:1074F4007FF410AF0123C360D0F8A4320BB103238F
:10750400C360022204F10C01204600F020F93D463C
:1075140003E74B88012B02D1C4F8A43206E0022B06
:107524007FF4F8AE8B881B0A80F8A032204600F066
:1075340038F9F2E690F89C32013B022BCAD84B880A
:10754400012B7FF4EAAE0023E6E700BF900600209B
:1075540070B50B7803F06002402A04460E4601D051
:107564005B061FD494F89C32013B022B1AD8317964
:107574000129204617D8FFF76CFE88B9D4F8B83231
:107584009B686BB1C4F8D40231462046984705463F
:10759400F3881BB915B9204600F003F9284670BDDD
:1075A4000325F5E72046FFF76AFE0025F6E770B5E8
:1075B4000B788A880E7903F06003202B04460D466D
:1075C40053D0402B51D063BB4B78012B3BD0032BC2
:1075D40020D033BB90F89C32022BD9B261D003295E
:1075E4001FD106F00F0312F0800F4FF0140202FBBC
:1075F400030365D09B8CA3B106F07F05013505EB31
:10760400850500EB850516F07F0365D12B6002220A
:10761400294651E090F89C32022BDAB237D0032A83
:1076240003D02046FFF72BFE0BE04B8833B97106DD
:1076340004D0EB8813B9314600F000FB204600F07B
:10764400B0F8002070BD90F89C32022BDAB21ED044
:10765400032AE6D14B88002BF3D1730602D03146BE
:1076640000F0F5FA204600F09CF831462046FFF77A
:10767400F2FD0028E5D1D4F8B832C4F8D4029B68EE
:10768400002BDED029462046BDE87040184772061C
:10769400C7D0314600F0D2FA8021204600F0CEFA5D
:1076A400CFE77106BDD113064CBF00F1140100F5FC
:1076B400AA7100230B600222204600F048F8C0E7BC
:1076C400B3F86431002BACD006F07F05142303FB20
:1076D400050505F5AA7596E73146204600F038FA07
:1076E40008B1012392E7286091E70B7803704B7887
:1076F40043704B8843808B888380CB88C3807047DA
:1077040010B58021044600F099FA20460021BDE816
:10771400104000F093BA30B588B1002401382346F4
:107724000134055D002DFAD1DBB201335B00138017
:107734000B7003234B70022310F8012F02B930BDE4
:10774400CA545A1CD2B202338D54DBB2F4E710B5DA
:1077540002241346C0E90622C0F894420A460021D6
:1077640000F087FA002010BD08B513460A46002130
:1077740000F07FFA002008BD10B503241346C0E9C9
:107784005622C0F894420A46002100F07BFA0020F9
:1077940010BD08B513460A46002100F073FA002014
:1077A40008BD08B504220023C0F8942219461A46DD
:1077B40000F05FFA002008BD08B505220023C0F8D8
:1077C400942219461A4600F05DFA002008BD000014
:1077D40008B50F490F480022FFF7B3FB08B1F9F7CA
:1077E40045FC0D490B48FFF7BFFB08B1F9F73EFC18
:1077F4000A490848FFF766FB08B1F9F737FC054862
:10780400FFF7CBFB18B1BDE80840F9F72FBC08BD62
:10781400B40000209406002018000020A0000020DE
:1078240000207047002070470020704737B5114B87
:107834000446186800909B880F48ADF80430FFF7A1
:1078440066FB6946204600F053FA50B12046F8F72B
:10785400D7FC05466846F8F7D3FC854201D1F9F711
:107864005FF94FF400620021204600F039FA00204D
:1078740003B030BD7C7D00089406002010B5064C92
:10788400064900222046FFF728FB05492046FFF75A
:1078940032FB002010BD00BF9406002070110020B0
:1078A40070090020122301480B807047E00000207B
:1078B400042301480B807047F40000200C23014886
:1078C4000B807047D4000020002370B54D1C1E4669
:1078D400040FB0F1204F34BF3034373401F8134073
:1078E40005F813600133DCB2A2424FEA0010EFD86E
:1078F40070BD00001A2310B50B800A4BD3F8100A90
:10790400D3F8182A80180AD0D3F8144A0649082252
:10791400FFF7DAFF042210312046FFF7D5FF0348B2
:1079240010BD00BF0070FF1FFA000020F800002007
:1079340010B5044C04480A462146FFF7ECFE2046E5
:1079440010BD00BF70190020827D000810B5044CE2
:1079540004480A462146FFF7DEFE204610BD00BF5C
:1079640070190020957D000810B5044C04480A469F
:107974002146FFF7D0FE204610BD00BF701900203D
:10798400AB7D000810B5044C04480A462146FFF7B5
:10799400C2FE204610BD00BF70190020B67D00084D
:1079A40030B59FB004461422002102A800F098F9D3
:1079B4005C22002107A800F093F92368B3F1A04FDB
:1079C40038D14FF4807307A80793FCF7B7FB08B1CD
:1079D400F9F74CFB184C194800250095236B43F02C
:1079E40001032363236B049503F0010300934FF415
:1079F400C052009B0223CDE9022303210A23CDE9CF
:107A0400051302A9FBF71EF8636B43F0800363635D
:107A14000195636C43F480436364636C03F48043B3
:107A2400019343202A462946019BFAF7D5FD4320BA
:107A3400FAF704FE1FB030BD0038024000000240D7
:107A440000F2C441D0F80805FFF7B9BA242303FBB8
:107A54000103D0F80805D3F88C22FFF7E0BA2423F9
:107A640003FB0103D0F80805DA6CFFF70DBBD0F86F
:107A74000805FFF7A7BBC16810B5044621B1022968
:107A840001D0F9F7F3FA0121D4F80805FFF782FBD6
:107A9400D4F80805BDE81040FFF74DBB10B5044607
:107AA400D0F80805FFF779FB2268D2F8003E43F0CE
:107AB4000103C2F8003E236A23B1034A136943F069
:107AC4000603136110BD00BF00ED00E0D0F8080507
:107AD400FFF76DBBD0F80805FFF795BBD0F8080594
:107AE400FFF77DBBD0F80805FFF7A1BBD0F8080568
:107AF400FFF79FBB08B5037802462BBB13484FF032
:107B0400A041C0F80825C2F8C8020622C0E9001244
:107B14000222C0E90323C0E90623C0E90833C0E90F
:107B24000B33FBF79FFC08B1F9F7A0FA8021074853
:107B3400FCF70CFA402200210448FCF7E7F903485B
:107B440080220121FCF7E2F9002008BD701B00200F
:107B540011F0800FD0F8C8324FF024021BBF01F09F
:107B64007F0102FB013102FB013191F83E0008BFA5
:107B740091F87E027047D0F8C802FBF7BCBD000044
:107B840010B5044611B1012916D010BD036A33B1F2
:107B9400F9F74CF9124A136923F0060313612268BA
:107BA400D4F80805D2F8003E23F00103BDE81040E4
:107BB400C2F8003EFFF7FBBA0268D0F80805D2F815
:107BC400003E43F00103C2F8003EFFF7E6FA236AE1
:107BD400002BDAD0024A136943F006031361D4E799
:107BE40000ED00E0004870477C2000207047000052
:107BF40003289ABF014B185C03207047C47D00081A
:107C040008B5D0F8C802FBF7B8FCBDE80840FFF798
:107C1400EFBF10B51446D0F8C8021A462346FBF746
:107C2400DFFCBDE81040FFF7E3BF08B5D0F8C80299
:107C3400FBF70EFDBDE80840FFF7DABF08B5D0F842
:107C4400C802FBF780FDBDE80840FFF7D1BF08B5C7
:107C5400D0F8C802FBF7AFFDBDE80840FFF7C8BF86
:107C640008B5D0F8C802FBF7A7FCBDE80840FFF749
:107C7400BFBF08B5D0F8C802FBF745FDBDE8084012
:107C8400FFF7B6BF08B5D0F8C802FBF710FDBDE892
:107C94000840FFF7ADBF000070B50D4D0D4C641BDF
:107CA400A4100026A64209D10B4D0C4C00F036F866
:107CB400641BA4100026A64205D170BD55F8043BF0
:107CC40098470136EEE755F8043B98470136F2E74A
:107CD400D07D0008D07D0008D07D0008D47D000848
:107CE40002440346934200D1704703F8011BF9E7AD
:107CF4000A7870B56AB970BD9A4209D10C46054636
:107D040014F8013F002BF6D015F8016F9E42F7D00E
:107D140001300378002BEFD11846ECE7F8B500BF2B
:107D2400F8BC08BC9E467047F8B500BFF8BC08BC58
:047D34009E467047B0
:107D3800EC000100C39000060101910000000A80D8
:107D48000000000493000001F40102030405060783
:107D580008090A00000000000000000001020304F6
:107D680006070809000000000102030400061016B7
:107D7800000610164D393939390053544D6963726C
:107D88006F656C656374726F6E6963730053544DED
:107D98003332205669727475616C20436F6D506F71
:107DA80072740043444320436F6E6669670043441E
:107DB8004320496E746572666163650000030103C0
:087DC8007C84FF7F0100000034
:047DD000E9010008BD
:047DD400C5010008DD
:107DD8000102030405060101010000000024F4006B
:107DE8000100000010000000F76D00089D6D0008FC
:107DF800956C0008000000001D6B00082D6C000841
:107E0800F56B000800000000000000000000000002
:107E1800AD6B0008616B0008A96B0008556B000882
:107E280009024300020100C03209040000010202F5
:107E380001000524001001052401000104240202A8
:107E48000524060001070582030800100904010043
:107E5800020A000000070501024000000705810230
:107E6800400000000A060002000000400100000077
:107E780081780008257800082978000831780008FA
:107E88002D780008A9780008B57800083579000829
:107E980051790008F97800086D7900088979000897
:107EA800C1780008050F0C0001071002020000004D
:107EB800120101020202004083044057000201023D
:107EC80003010000040309041A0300000000000075
:107ED800000000000000000000000000000000009A
:047EE8000000000096
:0400000508001EE9E8
:00000001FF
